:100000000C94D3030C94EE030C94EE030C94EE03C7
:100010000C94EE030C94EE030C94EE030C94EE039C
:100020000C94EE030C9451150C94EE030C94EE0317
:100030000C94AC280C94EE030C94EE030C94EE0399
:100040000C94EE030C94EE030C94EB130C94EE035F
:100050000C94F4080C94EE030C94BB080C94EE037F
:100060000C94571A0C94EE030C9467270C94EE032F
:100070000C944D5D0C94EE030C94EE03031BF61AE6
:10008000EA1AD01AB61A921AA41AD21D061D031D16
:10009000921AF01CD61CB61C961C441CF21B0F1B9B
:1000A000DC27CF271C280028F4278D279E279E2792
:1000B000A527C127BC27A127A927A527B827C5277A
:1000C000A127A927A527B427CA27A1272E280A0DCB
:1000D0003D3D3D3D3D3D3D3D3D3D3D3D3D3D3D3D50
:1000E0003D3D3D3D3D3D3D3D3D3D3D3D3D3D3D3D40
:1000F0003D3D3D000A0D466C69676874436F6E7440
:10010000726F6C0A0D48617264776172653A25649A
:100110002E25640A0D536F6674776172653A562511
:10012000642E2564256320000A0D47656E657261A3
:1001300074696E672064656661756C74204D6978BA
:100140006572205461626C65000A0D4D69786572B4
:100150002D436F6E6669673A20272573272028256F
:1001600075204D6F746F727329000A0D466F756E9E
:100170006420424C2D4374726C3A200025642000A8
:100180000A0D0A0D2121204D495353494E47204263
:100190004C2D4354524C3A202564202121000A0D55
:1001A0003D3D3D3D3D3D3D3D3D3D3D3D3D3D3D3D7F
:1001B0003D3D3D3D3D3D3D3D3D3D3D3D3D3D3D3D6F
:1001C0003D3D3D000A0D496E69742E204545505253
:1001D0004F4D003A2047656E65726174696E672005
:1001E00044656661756C742D506172616D657465EE
:1001F00072207573696E67206F6C64205374696335
:100200006B2053657474696E6773000A0D41434334
:10021000206E6F742063616C696272617465642022
:1002200021000A0D5573696E6720706172616D65FA
:10023000746572736574202564000A0D43616C69EE
:1002400062726174696E672070726573737572652E
:100250002073656E736F722E2E004F4B0A0D000ACD
:100260000D436F6E74726F6C3A200048656164696B
:100270006E67486F6C64004E6F726D616C20284130
:1002800043432D4D6F646529000A0D3D3D3D3D3DC5
:100290003D3D3D3D3D3D3D3D3D3D3D3D3D3D3D3D8E
:1002A0003D3D3D3D3D3D3D3D3D3D3D3D3D3D0A0DE1
:1002B000002E000A0D20444143206F722049324332
:1002C000204552524F522120436865636B204932CA
:1002D000432C2033567265662C2044414320616EC6
:1002E0006420424C2D4374726C005B25695D005B99
:1002F00025695D002B204D696B726F4B6F707465C3
:1003000072202B0048573A5625642E2564205357F7
:100310003A25642E256425630053657474696E67FD
:100320003A256420257300493243204552524F52EA
:10033000212121004D697373696E6720424C2D4362
:1003400074726C3A256421210028632920486F6C5F
:10035000676572204275737300486F6568653A205F
:100360002020202025356900536F6C6C486F65682C
:10037000653A20253569004C756674647275636B47
:100380003A20253569004F66662020202020203A3B
:1003900020253569004B65696E65200048F6686563
:1003A0006E726567656C756E6700616B742E204CAC
:1003B000616765004E69636B3A202020202020256C
:1003C000356900526F6C6C3A2020202020202535A2
:1003D00069004B6F6D706173733A20202025356979
:1003E000004B313A25346920204B323A25346920BC
:1003F000004B333A25346920204B343A25346920A8
:10040000004B353A25346920204B363A2534692093
:10041000004B373A25346920204B383A253469207F
:10042000004E693A2534692020526F3A25346920FC
:100430000047733A253469202047693A25346920FA
:100440000050313A253469202050323A2534692051
:100450000050333A253469202050343A253469203D
:10046000004779726F202D2053656E736F72004EB6
:1004700069636B2025346920282533692E25692975
:1004800000526F6C6C2025346920282533692E2595
:100490006929004769657220253469202825336958
:1004A00029004E69636B2025346920282533692E85
:1004B00025782900526F6C6C20253469202825335B
:1004C000692E25782900476965722025346920281E
:1004D00025336929004E69636B202534692028255E
:1004E000336929282533692900526F6C6C20253423
:1004F000692028253369292825336929004769653A
:100500007220253469202825336929282533692953
:1005100000414343202D2053656E736F72004E6976
:10052000636B2025346920282533692900526F6CBC
:100530006C2025346920282533692900486F6368B9
:1005400020253469202825336929005370616E6E97
:10055000756E673A202025356900456D70662E500E
:100560006567656C3A253569004B6F6D7061737313
:1005700020202020202020005269636874756E6757
:100580003A2020253569004D657373776572743A9A
:1005900020202535690053746172743A2020202090
:1005A0002025356900506F7469313A202025336960
:1005B00000506F7469323A202025336900506F74FF
:1005C00069333A202025336900506F7469343A202A
:1005D0002025336900536572766F202000536574BF
:1005E000706F696E742020253369005374656C6CDC
:1005F000756E673A202533690052616E67653A254A
:1006000033692D2533690045787465726E436F6ECA
:1006100074726F6C2020004E693A25346920205294
:100620006F3A253469200047733A25346920204702
:10063000693A253469200048693A25346920204305
:10064000663A2534692000424C2D4374726C204573
:1006500072726F727320002025336420202533646A
:100660002020253364202025336420002025336496
:100670002020253364202025336420202533642066
:100680000020253364202025336420202533642076
:10069000202533642000424C2D4374726C20666F19
:1006A000756E6420002025632020202563202020F3
:1006B000256320202025632000202563202020257D
:1006C000632020202563202020256320002025632F
:1006D0002020202D2020202D2020202D0031300012
:1006E0003131003132005069746368436F6E747247
:1006F0006F6C203120004D6F647573202020202006
:10070000202020203A202020253273005374616E6F
:100710006467617320202825303264293A2020251F
:1007200033690053636877656265676173202020D1
:10073000203A2020253369005069746368436F6E46
:1007400074726F6C20322000537469636B2D4465A2
:100750006C74612020203A202020253264000A0D8C
:10076000506C6561736520636F6E6E6563742053B2
:1007700070656B7472756D207265636569766572FC
:1007800020666F722062696E64696E67204E4F57F3
:100790002E2E2E006F6B2E0A0D0054696D656F753D
:1007A000742E0A0D000011241FBECFEFD0E1DEBF72
:1007B000CDBF13E0A0E0B1E0E6E3FCEC02C00590A1
:1007C0000D92AE3DB107D9F719E0AEEDB3E001C02F
:1007D0001D92A13CB107E1F70C9496040C94000023
:1007E0000E94025B0E94D05E0E94E85F0895282F5D
:1007F000FB018150853008F023E0842F99273327AF
:1008000021503040829FD001839FB00D929FB00D48
:100810001124AC59BF4F019724F00E94FD6501924D
:10082000FACF0895863038F085E0A2E0B0E0082ED7
:100830000E940A6608958823C1F70895582F8630CC
:1008400048F155E0842F9927252F33272150304038
:10085000829FD001839FB00D929FB00D1124AC599F
:10086000BF4FFB01019724F001900E940A66FACF66
:10087000A2E6B0E0042E0E940A66A0E5B0E088E09F
:10088000FB01182E0E941666852F0E9412040E94FA
:10089000025B08958823B1F60895CF93A2E0B0E0FB
:1008A0000E94FD65802DC82F8150853020F0C3E067
:1008B0008C2F0E9412048C2F9927CF91089580913C
:1008C0009008E82FFF27EE0FFF1FE25AF74F8081B5
:1008D00091818D5E9F4F14F0109202018081918171
:1008E0008A5B9F4F24F480910201882319F02091A4
:1008F0002B0715C081E08093020120912B07280F60
:1009000020932B07253038F088EE93E09093020473
:100910008093010404C0822F0E94E42BE8CF822F31
:1009200099279093F9078093F8070895CFEFD0E1C6
:10093000DEBFCDBF14B815B807EE13E00253104068
:1009400017FFFCCF08EE13E0189B6DC1199B76C111
:100950002DE02093010181E887B93E9A8FEF88B995
:100960008BE184B981E085B98EE38AB9579A87E42F
:100970008BB9469A84B7877F84BF80916000886175
:10098000809360001092600080ED97E090930204E5
:100990008093010410927104109270041092630805
:1009A00010926208109273041092720410927504EF
:1009B00010927404243108F43CC188E894E0A0E06B
:1009C000B0E08093850390938603A0938703B09350
:1009D00088032A3009F462C1243109F45FC1289ADE
:1009E0000E943A150E940A150E942B0E0E94972819
:1009F0000E9425190E9426270E94445778948EEC65
:100A000090E09F938F931F920E9456110F900F902A
:100A10000F9082E690E09F938F938DE090E09F93FC
:100A20008F9381E090E09F938F93809101016AE022
:100A30000E948D65892F99279F938F938091010143
:100A40000E948D6599279F938F9384EF90E09F93E9
:100A50008F931F920E9456118091C8002DB73EB708
:100A6000235F3F4F0FB6F8943EBF0FBE2DBF8032BD
:100A700009F40CC1809101018C3008F0D8C0299A8A
:100A800049E060E978E083E00E94F703C8EED3E034
:100A9000DE010E94FD65802D813009F4D1C088E21D
:100AA00091E09F938F931F920E9456110F900F9089
:100AB0000F9020E835E0F9018FE01586168617863D
:100AC000108A8150349687FFF8CF80E480938D059B
:100AD00080938E0510928F058093900580939105E9
:100AE00090EC9093920510929305809394058093D7
:100AF000950510929605909397059093980580938D
:100B0000990510929A0580939B0590939C0581E02E
:100B10008093800541E855E08BE0E3E0F1E0DA0105
:100B200001900D928A95E1F78DE4DE01F901182E0E
:100B30000E9416668091840399279F938F935F93F9
:100B40004F9389E491E09F938F931F920E945611D7
:100B50002DB73EB7295F3F4F0FB6F8943EBF0FBE8B
:100B60002DBF8AE691E09F938F931F920E945611AA
:100B700010924204109205040E94C4390F900F9005
:100B80000F90809105048823E1F310924204EE2433
:100B9000FF24ECE7CE2EE1E0DE2E109205040E9449
:100BA000C439809105048823E1F3F701EE5AF74F29
:100BB0008081882309F074C0E70121967E012C977B
:100BC00060F3EE24FF2470E8C72E71E0D72E22C018
:100BD000F701EE0FFF1FEE0FFF1FE058FA4F85855C
:100BE0001816F4F4E7012196DF93CF93DF92CF92AA
:100BF0009F930E9456110F900F900F900F900F909F
:100C000086E398E0E80EF91ED7011C927E012C972E
:100C100008F055C0F701EE5AF74F90819923C1F2C1
:100C2000E7012196EDCF199B2FC024E192CE2998A0
:100C300027CF8BE095E0A0E0B0E0C3CE2BE089CEDB
:100C4000A1E0B0E00E94FD65802D8F3F09F427CF21
:100C50001092840320E835E08DE4DE01F901182EBE
:100C60000E94056690918403F9013D962FE08081F2
:100C7000349618160CF49F5F215027FFF8CF9093FD
:100C8000840341E855E056CF2AE063CE8091CA0044
:100C9000863009F0EFCE0E94545CECCE2898A0CEAE
:100CA000E7012196DF93CF93DF92CF921F920E94AC
:100CB00056110F900F900F900F900F907FCF8EE9ED
:100CC00091E09F938F931F920E9456110F900F9067
:100CD0000F90A1E0B0E00E94FD65802D8B3409F0FB
:100CE00057C1A4E0B0E00E94FD65802D853008F07A
:100CF00037C20E944D044DE560E978E00E94F70399
:100D00000E944D0499279F938F9382E292E09F93D4
:100D10008F931F920E945611809198080F900F9008
:100D20000F900F900F9080FDF7C10E9420378091A7
:100D300001018A3009F4EEC1843109F4EBC1289A2B
:100D400080ED97E0909302048093010485E5809301
:100D50002D078FE592E09F938F931F920E9456116B
:100D6000809198080F900F900F9082FFF6C18BE64C
:100D700092E09F938F931F920E9456110F900F90B5
:100D80000F9089E892E09F938F931F920E945611D3
:100D90000E94F0030E949E1E88E893E19093A803AE
:100DA0008093A70381E080932C070F900F900F9002
:100DB00080910504882309F48EC08091180388234C
:100DC00009F489C01092050480912B07882309F447
:100DD0008AC00E945F040E94C439209101012A3018
:100DE00009F48AC0243109F487C0289A80910E033F
:100DF000882309F487C0815080930E038091760484
:100E0000882329F080917604815080937604809124
:100E10004E05882369F0815080934E05882341F464
:100E200010924C0510924B0510924A0510924905FC
:100E30008091A7039091A80301979093A8038093B2
:100E4000A7038091A7039091A803892B29F0809193
:100E50004104882309F465C08091A7039091A803F9
:100E6000892B09F464C080911103909112038F5F64
:100E70009F4F09F46CC080910504882321F0809174
:100E80006D04882311F40E94670E0E94530BC80161
:100E90000E94D7148823E9F08091A908282F3327CE
:100EA00080912603909127038217930744F4809141
:100EB0001103909112038F5F9F4F09F45CC00E9451
:100EC000E05984E08093000484E190E00E94CE1415
:100ED0008C010E94195B80910004882309F068CF7F
:100EE0000E94245A65CF0E94DE3D0E94C4392091A1
:100EF00001012A3009F076CF289880910E038823CB
:100F000009F079CF80933707109256041092550458
:100F100010925404109253041092520410925104EF
:100F20006DCF2A3031F1243121F1289AA4CF0E94CB
:100F30003C2785E090E09093A8038093A7038091DD
:100F40001103909112038F5F9F4F09F094CF80910E
:100F50006D04882309F48FCF80E197E29093020417
:100F60008093010480E890E0909312038093110332
:100F700082CF289880CF80E797E1909302048093F6
:100F8000010480E093E0909312038093110397CFC4
:100F90000E94BD2984EC91E09F938F931F920E9441
:100FA000561151E0952E0F900F900F90C0E5D0E0B4
:100FB0007E010894E11CF11C42E0C42ED12CCC0E21
:100FC000DD1E33E0A32EB12CAC0EBD1E24E0622E3C
:100FD000712C6C0E7D1E95E0492E512C4C0E5D1E21
:100FE00086E0282E312C2C0E3D1EE2E09E1609F4E0
:100FF0008BC0F3E09F1609F48AC023E0291508F49A
:1010000083C080910101843168F085E08093A80855
:101010001092C0088BE18093A4088EE48093BD08F1
:101020008093BE08DE010E94FD65802D8C3008F0A3
:1010300068C0D7010E94FD65802D8C3008F061C02A
:10104000D6010E94FD65802D8C3008F05AC0D50174
:101050000E94FD65802D8C3008F053C0DE010E9497
:10106000FD65802D80939008D7010E94FD65802D3D
:1010700080939108D6010E94FD65802D809392088F
:10108000D5010E94FD65802D80939308D3010E94B5
:10109000FD65802D80939408D2010E94FD65802D0E
:1010A00080939508D1010E94FD65802D809396085C
:1010B000A7E5B0E00E94FD65802D8093970831E0A0
:1010C000931651F483ED91E09F938F931F920E94AA
:1010D00056110F900F900F904DE560E978E0892D43
:1010E0000E941E04939495E0991508F07ECF83E04A
:1010F0000E9412048BE4A1E0B0E0082E0E940A6670
:10110000F0CD0E94A429E8CF0E946D2A7ACF0E94D8
:101110001F2B77CF289814CE8AE392E09F938F936A
:101120001F920E94561188EE93E00E94CE148C010B
:101130000E942B190F900F900F90C8010E94D71496
:101140008823D9F38AE592E09F938F931F920E94A0
:1011500056110F900F900F90E8CD87E792E009CEDF
:101160008BE092E09F938F931F920E9456110F90F5
:101170000F900F90BECD1F920F920FB60F921124B9
:101180008F939F93EF93FF93809110038823A9F48B
:101190008091F1039091F2030196FC01E352FA4F22
:1011A000E081ED3079F08639910561F09093F2039A
:1011B0008093F103E093C6000EC01092F2031092E8
:1011C000F10309C01092F2031092F10381E08093C1
:1011D0001003E093C600FF91EF919F918F910F90C4
:1011E0000FBE0F901F9018951F920F920FB60F927F
:1011F00011242F933F934F935F938F939F93AF93BC
:10120000BF93EF93FF9390E08091C6008093E90332
:101210005091F703563910F09093F8038091E90349
:101220008D3091F02091F803822F9927813091051C
:1012300009F46AC0823091050CF48CC0029709F45D
:101240007DC01092F803A6C02091F803223061F708
:101250009093F803852F9927865C984FFC0132976D
:1012600040812091F3033091F403241B3109DC0108
:1012700011978C91281B3109C9019F709093F40339
:101280008093F3030024880F991F001C880F991F77
:10129000001C892F902D982F935C9093F5032F734A
:1012A0003070235C2093F6038081891709F46CC0A9
:1012B00090E08091E6038F5F8093E6038091E803DE
:1012C000882309F067C0992309F464C081E0809302
:1012D000E803580F5093E5035150E52FFF27E65CD4
:1012E000F84F8DE0808380913C07823509F052C031
:1012F00088E190E02CE00FB6F894A8958093600008
:101300000FBE2093600046C02F5F2093F803E52FA7
:10131000FF27E65CF84F8091E90380835F5F50937D
:10132000F7032091E9038091F3039091F403820F76
:10133000911D9093F4038093F3032CC0E52FFF27B6
:10134000E65CF84F8091E9038083563938F31092B8
:10135000F803E7CF892B09F074CF8091E90383323A
:1013600059F08091E90380933A0781E08093F70375
:101370008091E9039927DDCF8091E803882389F7DD
:1013800081E08093F803EDCF8C91821709F090CF24
:1013900091E094CFFF91EF91BF91AF919F918F9189
:1013A0005F914F913F912F910F900FBE0F901F9023
:1013B0001895AC01A0E0B0E09D01A817B90748F46A
:1013C000EDEDF5E08191280F311D1196A417B507B9
:1013D000C8F33F70FD01E352FA4FC9010024880FA2
:1013E000991F001C880F991F001C892F902D835C6A
:1013F00080831196FD01E352FA4F2F733070822FD4
:10140000835C8083A252BA4F8DE08C9310921003BC
:101410008091DD058093C6000895BF92CF92DF9240
:10142000EF92FF920F931F93CF93DF93CDB7DEB769
:101430002C859D857E85BB2483E28093DD059F59A5
:101440009093DE052093DF0503E010E0772309F495
:10145000ADC0CF84D88843E1E42EF12CEC0EFD1E04
:10146000A989BA897150109709F4A0C0109709F49E
:101470003CC0F601EB0DF11DB3949081119789F4F6
:101480007723A1F1F70122E030E0E20EF31ED7014D
:10149000C080D180E20EF31E0D90BC91A02DBB2424
:1014A0007150109719F1F601EB0DF11DB3944081C5
:1014B000119709F466C01097D1F0F601EB0DF11DFC
:1014C000B39460811197A1F4772391F0F7013296DC
:1014D000D701CD90DC9032E0E32EF12CEE0EFF1E12
:1014E000A081B181BB24715003C090E040E060E076
:1014F000F801E352FA4F892F86958695835C8083A5
:101500000F5F1F4FF801E352FA4F892F992783701D
:10151000907082959295907F9827807F9827552785
:101520009A01329522952F7023273F702327822B13
:10153000835C80830F5F1F4FF801E352FA4F4F70B7
:101540005070440F551F440F551F862F99270024B4
:10155000880F991F001C880F991F001C892F902D40
:10156000842B835C80830F5F1F4FF801E352FA4F97
:101570006F73635C60830F5F1F4F109709F076CF26
:1015800015C0772309F4B3CFF701A2E0B0E0EA0E6B
:10159000FB1ED701C080D18022E030E0E20EF31EB6
:1015A0000D90BC91A02DBB24715085CFC8010E9425
:1015B000D909DF91CF911F910F91FF90EF90DF90AC
:1015C000CF90BF900895A3E07A2F4091E503465055
:1015D00009F45FC0E72FFF27E65CF84F80818D5349
:1015E0007F5FE72FFF27E65CF84F20812D537F5F59
:1015F000E72FFF27E65CF84F30813D537F5FE72FF1
:10160000FF27E65CF84F60816D537F5F9927880F55
:10161000991F880F991F522F52955F70582B822F58
:1016200099278F70907082959295907F9827807FF0
:101630009827232F26952695282B832F992783706B
:1016400090700024969587950794969587950794B2
:10165000982F802D682B41504F3FD9F0EA2FFF275C
:10166000E65CF84F5083AF5F41504F3F91F0EA2F57
:10167000FF27E65CF84F2083AF5F41504F3F49F0B2
:10168000EA2FFF27E65CF84F6083AF5F442309F041
:10169000A1CF8DE397E09093E4038093E303A350FD
:1016A000A093E2030895CF93DF93CDB7DEB72297DF
:1016B0000FB6F894DEBF0FBECDBF8091E80388233C
:1016C00009F4ACC20E94E30A80913B07823609F418
:1016D00071C080913C0799278436910509F457C061
:1016E0008536910584F58136910509F44EC182361F
:1016F00091050CF4C2C08236910509F49AC1833673
:101700009105C1F48091DE039091DF03892B09F0EC
:101710004CC2A091E303B091E4039C91992309F09A
:101720003AC29C918AE0989FC00111249093DF03F4
:101730008093DE031092E8031092E4031092E30317
:101740001092E2036BC28C36910509F410C18D36FC
:1017500091050CF0B3C08736910509F42BC188368A
:10176000910541F78FEF80930E03E091E303F09131
:10177000E403808190913C04892B80933C0488236E
:1017800011F01092EA0381E08093EE03D3CFE09151
:10179000E303F091E40390818AE0989FC001112453
:1017A00090930C0380930B03892B21F281E08093AB
:1017B000ED03C0CF80913C0799278037910509F44C
:1017C000F2C0813791050CF485C08337910509F487
:1017D0005BC1843791050CF03CC18137910509F05C
:1017E00078CFA091E303B091E4038C918F3F09F48B
:1017F00009C28C91882309F000C281E08C93A091EA
:10180000E303B091E4034DE560E978E08C910E9438
:10181000F703809110038823E1F3E091E303F09153
:10182000E403808189838BE48A838DE590E09F9334
:101830008F9380E998E09F938F9321E030E03F936E
:101840002F93CE0102969F938F933F932F93CE01B8
:10185000820F931F9F938F9383E08F9381E08F93E9
:1018600081E58F930E940D0AADB7BEB71F960FB6E4
:10187000F894BEBF0FBEADBF2CCF8B34910509F0DD
:1018800059CFE091E303F091E4038081918190933B
:101890008904809388042091860430918704821BF8
:1018A000930B845E9D4F68E671E00E94AD65845B9A
:1018B000904090938504809384043CCF84379105B5
:1018C00009F47CC08637910509F034CF81E080931C
:1018D000EC0330CF8D36910529F18E3691050CF051
:1018E00093C08B34910509F0F4CEA091E303B0913D
:1018F000E4038D919C9190938904809388042091B6
:10190000860430918704821B930B845E9D4F68E6AA
:1019100071E00E94AD65845B904090938504809354
:101920008404D7CE809110038823E1F3A091E303D0
:10193000B091E4039C91913009F43CC1198281E09B
:1019400090E09F938F93CE0101969F938F9381E0B8
:101950008F938F938DE48F930E940D0A8DB79EB75E
:1019600007960FB6F8949EBF0FBE8DBFB2CE8FEF15
:1019700080930E03E091E303F091E4038081809370
:101980003D0481E08093EF03D5CEE091E303F09135
:10199000E403E081E03258F08FE180930F038FEF92
:1019A00080930E03C7CE81E08093EB0392CEE09349
:1019B0000F03F5CF81E08093F003BCCE8091E50367
:1019C000853108F4D7C0E091E303F091E40380E1AE
:1019D000A5E1B7E001900D928A95E1F7809110039F
:1019E0008823E1F31F9280910D038F9384E58F93F9
:1019F0000E940D0A8AEF8093E0038FEF80930E031D
:101A00000F900F900F9096CE8E36910509F061CE13
:101A1000809110038823E1F38DE490E09F938F93EE
:101A200080E895E09F938F9381E08F938F938EE46E
:101A300092CFA091E303B091E4038BE0EDE2F7E0F5
:101A40000D9001928A95E1F78091360780931208F4
:101A5000A6CF8437910509F03CCE8091E50385310E
:101A600008F4B9C0A091E303B091E40380E1E5E19B
:101A7000F7E00D9001928A95E1F780EF8093E00303
:101A80008FEF80930E0325CE2091E3033091E40382
:101A9000F90180818150853018F481818B34E9F01F
:101AA0001982809110038823E1F381E090E09F93F5
:101AB0008F93CE0101969F938F9381E08F938F93A5
:101AC00083E58F930E940D0AEDB7FEB737960FB6E8
:101AD000F894FEBF0FBEEDBFFCCD60E978E08DE568
:101AE0002E5F3F4FDB01F901982F01900D929A95DF
:101AF000E1F722503040482FD9018C910E941E04FA
:101B00008091BD089927AA27BB27BC01CD0124ECF1
:101B100039E040E050E00E946E65DC01CB0180932B
:101B2000A1039093A203A093A303B093A403809175
:101B3000BE089927AA27BB27BC01CD010E946E656C
:101B4000DC01CB0180939D0390939E03A0939F03A0
:101B5000B093A003E091E303F091E40380810E943D
:101B600012040E944D0489830E94F00389810E941F
:101B7000E42B97CFE091E303F091E403808191811E
:101B8000A281B3818093150790931607A09317073E
:101B9000B093180723CF8AE0989FC00111240E94B8
:101BA000CE149093DC058093DB05A091E303B09104
:101BB000E403B7CD40E855E08DE4FA01282F0D90FD
:101BC00001922A95E1F7A8EEB3E0FA01182E0E94DF
:101BD00016669983B4CEA091E303B091E4038D918E
:101BE0009D910D90BC91A02D8093150790931607A1
:101BF000A0931707B093180740CF863008F403CEA0
:101C000085E0FCCD0E944D04E091E303F091E403F4
:101C10008083A091E303B091E403EBCD22960FB64D
:101C2000F894DEBF0FBECDBFDF91CF910895CF9363
:101C3000C82F8A3029F08091C00085FFFCCF04C0F6
:101C40008DE00E94170EF7CFC093C60080E090E0B1
:101C5000CF910895089588E18093C1008091C000DC
:101C600082608093C0008091C10080688093C10031
:101C70008091C10080648093C1008AE28093C40097
:101C800080910B0390910C030E94CE1490930A074D
:101C9000809309078CED90E00E94CE149093390751
:101CA0008093380710920B078AE480930C0784E036
:101CB00080930F078AE080930D0781E080930E07E1
:101CC0001092E4031092E3031092E2030895EF925E
:101CD000FF920F931F9380911003882309F478C219
:101CE0008091EE03882309F082C08091EF0388235E
:101CF00029F080911003882309F07FC18091EC03C3
:101D0000882329F080911003882309F05BC180911A
:101D1000F003882329F080911003882309F036C14D
:101D200080913807909139070E94D714882329F0B1
:101D300080911003882309F0C8C080910B03909113
:101D40000C03892B09F084C18091ED03882329F0CD
:101D500080911003882309F00FC28091DE039091D7
:101D6000DF03892B09F07EC120910F032F3F59F12A
:101D700080E190E09F938F93822F9927829592958F
:101D8000907F9827807F9827855F9E4F9F938F93A2
:101D900081E090E09F938F938FE093E09F938F93E8
:101DA00082E08F9381E08F9381E48F930E940D0AEC
:101DB0008FEF80930F038DB79EB70B960FB6F894F5
:101DC0009EBF0FBE8DBF80911208882329F080919D
:101DD0001003882309F05EC08091EB03882309F487
:101DE000F7C180911003882309F4F2C139C08091B2
:101DF0001003882309F479CF0E94A71E84E190E0A4
:101E00009F938F939091EA0384E1989FC0011124DE
:101E1000875D9C4F9F938F9381E090E09F938F937A
:101E20008AEE93E09F938F9382E08F9381E08F936C
:101E300088E48F930E940D0A8091EA038F5F2DB78B
:101E40003EB7255F3F4F0FB6F8943EBF0FBE2DBF84
:101E5000843008F4B8C11092EA031092EE0345CF23
:101E600086E190E09F938F938EE598E09F938F9308
:101E700081E08F938F9380E58F930E940D0A1092DB
:101E8000EB038DB79EB707960FB6F8949EBF0FBEB3
:101E90008DBF9EC181E090E09F938F9382E198E097
:101EA0009F938F9381E08F938F9382E48F930E940F
:101EB0000D0A109212082DB73EB7295F3F4F0FB69B
:101EC000F8943EBF0FBE2DBF87CF8091A4089927FD
:101ED000880F991F880F991F7C010027F7FC009538
:101EE000102F8091C2049091C304A091C404B091BA
:101EF000C504BC01CD01A80197010E94E2653093A1
:101F00002607209325078091BA049091BB04A091E5
:101F1000BC04B091BD04BC01CD01A80197010E9491
:101F2000E265309328072093270780915E04809311
:101F3000290780915D0480932A0788E090E09F93B1
:101F40008F9385E297E09F938F9381E08F9383E057
:101F50008F9387E78F930E940D0A80912B072DB7EF
:101F60003EB7295F3F4F0FB6F8943EBF0FBE2DBF5F
:101F7000853018F086E080932B0783E690E00E947E
:101F8000CE149093390780933807D7CE8BE090E03A
:101F90009F938F938DE297E09F938F9381E08F9330
:101FA00080910D038F9387E48F930E940D0A109206
:101FB000F0038DB79EB707960FB6F8949EBF0FBE7D
:101FC0008DBFAECE8AE090E09F938F938BE097E039
:101FD0009F938F9381E08F938F9386E58F930E94D9
:101FE0000D0A1092EC032DB73EB7295F3F4F0FB695
:101FF000F8943EBF0FBE2DBF8ACE0E94A71E80E57B
:1020000090E09F938F9389E293E09F938F9321E0D9
:1020100030E03F932F9388E293E09F938F933F9319
:102020002F938DE394E09F938F9383E08F9381E0D0
:102030008F938CE48F930E940D0A1092EF038DB75B
:102040009EB70F960FB6F8949EBF0FBE8DBF56CEAB
:102050008091090790910A070E94D714882309F0FC
:1020600077CE72CE8091DB059091DC050E94D7146B
:10207000882309F479CE80911003882309F474CE63
:102080008091A4089927880F991F880F991F7C01B8
:102090000027F7FC0095102F8091C2049091C30493
:1020A000A091C404B091C504BC01CD01A801970161
:1020B0000E94E2653093CE052093CD058091BA044D
:1020C0009091BB04A091BC04B091BD04BC01CD01B2
:1020D000A80197010E94E2653093D0052093CF05B7
:1020E0002091540930915509409156095091570952
:1020F000DA01C90103E0880F991FAA1FBB1F0A95C7
:10210000D1F7820F931FA41FB51F820F931FA41F27
:10211000B51F20918503309186034091870350912C
:102120008803BC01CD010E94E2653093D205209363
:10213000D1058EE090E09F938F938DEC95E09F9377
:102140008F9381E08F938F9383E48F930E940D0A86
:102150008091DE039091DF030E94CE149093DC0502
:102160008093DB052DB73EB7295F3F4F0FB6F8943C
:102170003EBF0FBE2DBFF8CD82E490E09F938F93BA
:1021800080ED97E09F938F9381E08F938F9384E40A
:102190008F930E940D0A1092ED038DB79EB707969C
:1021A0000FB6F8949EBF0FBE8DBF80910B03909128
:1021B0000C03009709F4D1CD0E94CE1490930A0726
:1021C00080930907CACD8093EA031092EE038DCD68
:1021D0001F910F91FF90EF900895982F8091130811
:1021E000813031F0892F0E94170E282F33270CC021
:1021F00080913E04E82FFF27E75DFC4F90838F5FBF
:1022000080933E0421E030E0C90108950F931F93AD
:10221000CF93DF938C01EB01672B71F0F801819173
:102220008F010E94ED10219739F0F80181918F0103
:102230000E94ED10219791F7DF91CF911F910F919F
:1022400008950F931F93CF93DF938C01EB01672BBE
:1022500081F0F8010F5F1F4F84910E94ED102197CC
:1022600041F0F8010F5F1F4F84910E94ED102197FC
:1022700081F7DF91CF911F910F910895CF93C82FD0
:10228000181634F480E20E94ED10C1501C16D4F3ED
:10229000CF910895CF93C82F181634F480E30E948D
:1022A000ED10C1501C16D4F3CF9108952F923F9298
:1022B0004F925F926F927F928F929F92AF92BF9256
:1022C000CF92DF92EF92FF920F931F93CF93DF9302
:1022D000CDB7DEB7E0970FB6F894DEBF0FBECDBF27
:1022E00026968FAD26972896EEADFFAD28978824C9
:1022F000992454018093130848E4C42ED12CCC0EA9
:10230000DD1E7F01C701F7011491112331F0153251
:1023100021F00894E11CF11CF6CFB701681B790B82
:1023200009F095C0112309F43DC20894E11CF11C89
:102330001FA63FA4232C0FEF39A6F7010894E11C38
:10234000F11C14911537C9F1812F80628837A9F1EA
:10235000103209F440C0133209F48DC01A3209F466
:1023600079C01D3209F476C01B32C9F11E32C9F1A1
:10237000103309F48AC0812F8153893008F07EC060
:1023800060E070E0CB01880F991F880F991F880FBC
:10239000991F860F971F680F791F610F711D60537A
:1023A0007040F7010894E11CF11C1491812F8053B7
:1023B0008A3040F3262E153739F630FE3DC0F6013F
:1023C00084E090E0C80ED91E80809180A280B38006
:1023D000103209F0C0CF89A5882309F0AECF19A724
:1023E000ACCFF7010894E11CF11C14911A3209F4E6
:1023F00051C060E070E014C0CB01880F991F880FB6
:10240000991F880F991F860F971F680F791F610FFB
:10241000711D60537040F7010894E11CF11C149188
:10242000812F80538A3040F3EFEF6F3F7E0714F423
:102430006FEF7FEF062F86CFF60182E090E0C80EA7
:10244000D91E808191814C01AA24BB2481CF0E9496
:10245000211168CF1A3251F4F60182E090E0C80EE3
:10246000D91E208022200CF068CF219490E1392AD7
:10247000EFED3E2262CF98E0392A5FCF1836C9F0DF
:102480001C36D1F481E0382A58CF34FC56CFF0E224
:102490003F2A53CFF60182E090E0C80ED91E60813A
:1024A00071819FEF6F3F790714F46FEF7FEF062F75
:1024B00044CF24E0322A41CF133609F44DC11434FD
:1024C00009F41FC1143609F41CC1193609F419C1E5
:1024D0001F3409F40FC11F3609F40CC1103709F479
:1024E000F9C0133709F4B2C0153509F4ECC015373B
:1024F00009F4E9C0183509F444C0183709F441C09B
:10250000112309F44FC1CE0101969DA78CA7198311
:1025100081E0482E19A6632C7724042D5FA454185B
:1025200057FC2DC029A5222331F10F5F050DC301F2
:1025300080739070892B09F42FC1222309F027C1E1
:1025400066FC1BC1C30180739070809709F410C1B1
:10255000852D0E944A11842D992787FD9095BC01F5
:102560008CA59DA50E94061164FECCCE822D801BF9
:102570000E943E11C7CE66FED9CF0E5FD7CF55243D
:10258000D1CFE0E1EEA733FE07C081149104A1048E
:10259000B10411F0F0E43F2A19A60FA707FD02C00D
:1025A0002FED3222CE0189969DA78CA7811491042C
:1025B000A104B10419F49FA5992361F1EEA54E2E53
:1025C00055246624772418AA84149504A604B70415
:1025D00010F0F1E0F8ABC501B401A30192010E9433
:1025E000C065DC01CB01082F8A30F0F4005DECA55A
:1025F000FDA50293FDA7ECA7C501B401A3019201BB
:102600000E94C06549015A01F8A9FF23E1F62EA5F1
:10261000283079F0632C7724CE010196482EFCA552
:102620004F1A28E2420E79CF095A183501F70F7D6B
:10263000DECF632C772463FEEFCF003369F380E3B2
:10264000ECA5FDA58293FDA7ECA7E6CFF60182E0FD
:1026500090E0C80ED91E0190F081E02DFDA7ECA7F7
:10266000EF2B81F4FE013196FDA7ECA788E2898368
:102670008EE6818385E78B838CE68C838D8389E26C
:102680008E831F8207FD15C0802F992787FD9095A7
:10269000AC0160E070E08CA59DA50E948764009766
:1026A00031F0482EFCA54F1A04150CF033CF402E04
:1026B00031CFECA5FDA501900020E9F731974E2E12
:1026C0002CA5421A27CF153511F481E0382A9AE05B
:1026D0009EA762CFF60182E090E0C80ED91E8081ED
:1026E00091814C01AA24BB2490E19EA7E0E43E2AFC
:1026F00018E752CF1F3411F4E1E03E2AF8E0FEA7BC
:102700004BCF143411F491E0392A30FE18C0F60191
:1027100084E090E0C80ED91E80809180A280B380B2
:10272000B7FE0AC0B094A09490948094811C911C30
:10273000A11CB11C8DE289A79AE09EA72ECFF601BD
:1027400082E090E0C80ED91E808191814C01AA24BC
:1027500097FCA094BA2CE4CFFE013196FDA7ECA71C
:10276000F60182E090E0C80ED91E80818983D0CE28
:10277000822D801B0E944A11EBCE80E38AA71BA703
:1027800062E070E0CE018A960E940611DBCE61E025
:1027900070E0CE018996F8CF822D801B0E943E11F9
:1027A00029A5CBCEE0960FB6F894DEBF0FBECDBF05
:1027B000DF91CF911F910F91FF90EF90DF90CF901D
:1027C000BF90AF909F908F907F906F905F904F9051
:1027D0003F902F9008951F920F920FB60F921124E1
:1027E0002F933F935F936F937F938F939F93AF93B9
:1027F000BF93EF93FF9380910004882329F0809189
:1028000000048150809300048091080481508F3F20
:1028100009F493C08093080480910104909102040C
:10282000029700F180910104909102040197909326
:10283000020480930104809101049091020420918C
:1028400011033091120382239323892B89F0809105
:1028500001018A3009F48BC0479A8091980883FF60
:102860008DC010C08FEF9FEF9093120380931103E0
:10287000809101018A3009F478C0479880919808C6
:1028800083FF7CC086B19927FC01E071F07084FF62
:102890000AC080910304909104040196909304046B
:1028A000809303046BC08091030490910404892BEE
:1028B00049F180910304909104048A56914010F5E7
:1028C000809103049091040469E270E00E9499658C
:1028D0008091030490910404860F971F9093040441
:1028E0008093030480910304909104040B9708F4EF
:1028F00040C080910304909104040A979093890446
:1029000080938804809188049091890420918604A2
:1029100030918704821B930B845E9D4F68E671E0C3
:102920000E94AD65845B90409093850480938404FD
:10293000109204041092030421C089E080930804DB
:10294000809113038F5F817080931303882319F4A0
:1029500081E080930504809106049091070401961C
:10296000909307048093060457CF5A9887CF5A9ABA
:1029700085CFF0938904E0938804C4CFFF91EF9151
:10298000BF91AF919F918F917F916F915F913F9197
:102990002F910F900FBE0F901F9018952091060455
:1029A00030910704280F391FC9010196089520911D
:1029B000060430910704821B930B892F9927869573
:1029C000807490700895CF93DF930E94CE14EC0131
:1029D000CE010E94D7148823D9F3DF91CF910895B7
:1029E0001F93CF93DF930E94CE14EC011FEC08C01D
:1029F00080911803882321F09093180310937A0094
:102A0000CE010E94D714982F882391F3DF91CF91A4
:102A10001F9108959FB7F894579A5F983E9A469AE7
:102A20008091B0008F708093B0008091B00083607F
:102A30008093B0008091B1008B738093B10080913E
:102A4000B1008B608093B1001092B2008FEF809341
:102A5000B3008091B00080688093B00080917000D6
:102A60008A7F8093700080917000826080937000F4
:102A70009FBF08958AE090E00E94CE1490931004C6
:102A800080930F0482E085BD83EA84BD17BC88E78C
:102A900088BD86E086BD80916E00816080936E0067
:102AA00008951F920F920FB60F9211242F933F9308
:102AB0004F935F936F937F938F939F93AF93BF9346
:102AC000CF93DF93EF93FF93809101018431C0F4A2
:102AD00080910904882309F446C020910A043091AA
:102AE0000B0441E02F37340708F4CAC08FEF8093FE
:102AF000B3002F5F304030930B0420930A0492C33D
:102B000080910904882349F78091B00086FFDBC0DB
:102B10008091B0008F7B8093B000E0910E04EE2393
:102B200009F01CC18091B608282F33278DED96E05F
:102B3000289FA001299F500D389F500D1124CA01D4
:102B400020910C0430910D04821B930B90930B0485
:102B500080930A0410920D0410920C04469A81E0AE
:102B600080930904BACF8091B00086FFD5C08091D0
:102B7000B0008F7B8093B00089EA93E090930B04C0
:102B800080930A048091B4089927880F991F880FB1
:102B9000991F2091FD033091FE032817390754F047
:102BA0008091B5089927880F991F880F991F821760
:102BB000930724F49093FE038093FD038091C5084E
:102BC00080FF70C1C091C204D091C304E091C404DD
:102BD000F091C5048091BA049091BB04A091BC040B
:102BE000B091BD04C81BD90BEA0BFB0B80911403F9
:102BF00090911503BC01660F771F680F791F8091B4
:102C000090039927880F991F880F991F680F791FC4
:102C100077FD21C2CB0195958795959587959093E2
:102C20001503809314039093FC038093FB0380911E
:102C3000DC0880FFD9C08091B308682F77278827E8
:102C400099279E01AF01F7FDEDC1A7E05595479586
:102C500037952795AA95D1F70E946E659B01AC0127
:102C600097FD03C2F6E05595479537952795FA9558
:102C7000D1F78091FB039091FC03820F931FD8C082
:102C80002F3F310569F060F0A9014F5F50404F3789
:102C9000510588F480E88093B300205830402BCF52
:102CA00080910A048093B30010920B0410920A04DE
:102CB00010920904B7C28FEF8093B30050930B04B6
:102CC00040930A04AFC28091B00080648093B0004A
:102CD0008CEB90E090930B0480930A0480910C0499
:102CE00090910D0484549F4F90930D0480930C0495
:102CF0008091FF03882329F080917604853B08F0BA
:102D0000DAC090910E049F5F8091B608891708F091
:102D100068C010920E0423CF8091B000806480932D
:102D2000B0008091B608282F33278DED96E0289FBC
:102D3000A001299F500D389F500D1124CA012091E8
:102D40000C0430910D04821B930B90930B04809321
:102D50000A049C0181E080930904C3CE89EA93E0D0
:102D600090930B0480930A048E2F9927813091054C
:102D700009F4A3C0029709F47DC1FF27EE0FFF1FDE
:102D8000E25AF74F80819181880F991F20910A04A0
:102D900030910B04820F931F90930B0480930A04CD
:102DA00020910A0430910B0455E02D3D350708F4BD
:102DB00045C18CED95E090930B0480930A049C012F
:102DC0002C5B304030930B0420930A0480910C0458
:102DD00090910D04820F931F90930D0480930C0427
:102DE000BECE90930E04BBCE8091B308682F772798
:102DF000882799279E01AF01F7FD0FC1E7E05595A0
:102E0000479537952795EA95D1F70E946E659B0106
:102E1000AC0197FD25C176E05595479537952795E7
:102E20007A95D1F78091FB039091FC03821B930B61
:102E30009093FC038093FB032091FB033091FC03F0
:102E400080910A0490910B04280F391F20503240C2
:102E50008091FB039091FC0397FD00C195958795A8
:102E6000959587959093FC038093FB038091FB03DA
:102E70009091FC039093FB078093FA0745E02D3D6A
:102E8000340708F4D4C08CED95E090930B04809344
:102E90000A0420910A0430910B0430930D0420930E
:102EA0000C0458CFC091C204D091C304E091C40473
:102EB000F091C5049BCE469824CF80911403909145
:102EC00015039C01220F331F280F391F8091900397
:102ED0009927880F991F880F991F280F391F37FDD1
:102EE0007BC1C90195958795959587959093150315
:102EF000809314039093FC038093FB038091C50897
:102F000080FF3CC12091C2043091C3044091C404AD
:102F10005091C5048091BA049091BB04A091BC0467
:102F2000B091BD04281B390B4A0B5B0B8091DC0868
:102F300080FF2DC18091B308682F772788279927B4
:102F4000EA01D90157FD5FC127E0D595C795B7952F
:102F5000A7952A95D1F79D01AE010E946E659B0150
:102F6000AC0197FD4BC1F6E05595479537952795F0
:102F7000FA95D1F78091FB039091FC03820F931F88
:102F80009093FC038093FB038091B408282F332790
:102F9000220F331F220F331F8091FB039091FC03FC
:102FA000821793077CF08091B508282F3327220FD2
:102FB000331F220F331F8091FB039091FC032817CE
:102FC000390724F43093FC032093FB038091FB0327
:102FD0009091FC0320910A0430910B04820F931FFF
:102FE0008050924090930B0480930A048091FB03DD
:102FF0009091FC0397FDEEC09595879595958795E3
:103000009093FC038093FB038091FB039091FC035E
:103010009093FB078093FA07C3CE21583F4F4F4F41
:103020005F4FECCE21583F4F4F4F5F4F0ECE51E0D8
:103030002737350758F487E791E027CF81E0273716
:10304000380708F0BDCE87E791E0B5CE30930B048A
:1030500020930A041ECF6D5F7F4FDCCD0396FECE1A
:10306000215C3F4F4F4F5F4FD6CE215C3F4F4F4FBC
:103070005F4FF8CD80911603909117039C01220FAA
:10308000331F280F391F205C3E4F37FDB4C0C901E4
:10309000959587959595879590931703809316033B
:1030A0009093FA038093F9036091BA047091BB0482
:1030B0008091BC049091BD0497FD98C0F7E0959570
:1030C000879577956795FA95D1F728EC30E040E041
:1030D00050E00E946E6597FD84C0272F382F492F3E
:1030E000552747FD5A958091F9039091FA03820F75
:1030F000931F9093FA038093F9038091B408282FCB
:103100003327220F331F220F331F8091F903909131
:10311000FA03821793077CF08091B508282F332794
:10312000220F331F220F331F8091F9039091FA036E
:103130002817390724F43093FA032093F903809178
:10314000F9039091FA0320910A0430910B04820F45
:10315000931F8050924090930B0480930A048091B7
:10316000F9039091FA0397FD3AC095958795959547
:1031700087959093FA038093F90312CE2091C204AD
:103180003091C3044091C4045091C504CFCE8091C6
:10319000B308682F77278827992757FD3EC0E7E0B7
:1031A0005595479537952795EA95D1F70E946E6515
:1031B0009B01AC0197FD2CC066E05595479537956E
:1031C00027956A95D1F78091FB039091FC03821BB0
:1031D000930BD6CE039610CF2D5F3F4F82CE039632
:1031E000C4CF61507F4F8F4F9F4F77CF61587F4F34
:1031F0008F4F9F4F63CF2D5F3F4F49CF215C3F4F94
:103200004F4F5F4FB0CEA158BF4FCF4FDF4F9CCE37
:10321000215C3F4F4F4F5F4FCFCF21583F4F4F4F14
:103220005F4FBDCFFF91EF91DF91CF91BF91AF91F4
:103230009F918F917F916F915F914F913F912F91CE
:103240000F900FBE0F901F90189510927C008FEC7E
:1032500080937A000895EF92FF920F931F93CF937C
:10326000DF9303E010E0D8010E94FD65802DC82F98
:10327000DD27C531D10508F02A97C7BD1092180483
:1032800084E690E00E94F01480911C0390911D034D
:103290008255934010F4C0E0D0E0CA3FD105E0F47D
:1032A00081EBE82E82E0F82EC7BD82E390E00E9419
:1032B000F014FF92EF921F920E94561180911C030E
:1032C00090911D030F900F900F908255934020F026
:1032D0002196CA3FD10540F3D8010C2E0E940A6600
:1032E000C09321088CE291E00E94F014DF91CF910D
:1032F0001F910F91FF90EF900895EF92FF920F931F
:103300001F93CF93DF9300E0009313040093120404
:103310000093110480ED97E00E94CE14EC011CE8AC
:1033200021E0F22E95EFE92E033009F4ABC000E066
:1033300080912404909125048C5F93400CF091C0FF
:1033400080911B03815080931B03809122049091F4
:1033500023048C5F93400CF079C080911A03815054
:1033600080931A0380912004909121048C5F9340F4
:103370000CF04AC08091190381508093190388E0B2
:10338000809344040E942C2780911B038A3008F00C
:1033900055C0F09213048AE080931B0380911A03B6
:1033A0008A3008F043C0F09212048AE080931A0336
:1033B000809119038A3098F5F09211048AE0809385
:1033C000190380914404882379F0CE010E94D71418
:1033D0008823B9F383EB92E09F938F931F920E940F
:1033E00056110F900F900F9010921C088FEC809345
:1033F0007A0080911C088823E1F31A3008F447C052
:10340000115009F091CF48C080912004909121047F
:10341000875094408CF1809119038F5FAECF863F27
:1034200080F2F0921104E0921903CBCF863F08F4AA
:10343000BFCFF0921204E0921A03BACF863F08F48D
:10344000ADCFF0921304E0921B03A8CF8091220429
:1034500090912304875094408CF080911A038F5FE1
:103460007FCF80912404909125048750944044F0AC
:1034700080911B038F5F67CF0F5F81CF0F5F72CF8C
:1034800001E063CF1B3008F452CF19E050CF8AE03F
:1034900090E00E94F014B4CF86E490E00E94F01413
:1034A000DF91CF911F910F91FF90EF9008951F92A0
:1034B0000F920FB60F921124EF92FF920F931F936A
:1034C0002F933F934F935F936F937F938F939F932C
:1034D000AF93BF93CF93DF93EF93FF9320912D048E
:1034E000822F9927AA27BB272F5FFC01429740F420
:1034F000E25CFF4FEE0FFF1F0590F491E02D099461
:1035000010922D0482E080932C0480912C048093EF
:103510007C0080912D04882309F4F9C38FEC8093FB
:103520007A00F5C320932D04809178009091790062
:103530002091320430913304820F931F909333040F
:103540008093320481E0DFCF20932D0480917800B6
:10355000909179002091300430913104820F931FB3
:10356000909331048093300484E0CDCF20932D04D8
:1035700080917800909179002091D0043091D1040D
:10358000821B930B9093200880931F0880911F0843
:103590009091200890933B0480933A0482E0B3CF4B
:1035A00020932D048091CE049091CF042091780037
:1035B00030917900821B930B909315088093140827
:1035C00080911408909115089093390480933804E1
:1035D00087E099CF20932D04809178009091790015
:1035E00090932F0480932E0486E08DCF20932D049A
:1035F0002091780030917900309331042093300489
:1036000010922C0482CF20932D04209178003091C9
:103610007900309333042093320481E074CF109208
:103620002D0481E080931803809114049091150477
:1036300001969093150480931404809178009091E2
:1036400079002091240830912508820F931F9093D0
:1036500025088093240880911C088F5F80931C08A4
:1036600080911C08853008F44DCF809124089091FA
:10367000250897FD36C395958795909325088093E7
:103680002408809178009091790090931D03809395
:103690001C0310921C088091160490911704BC0121
:1036A000660F771F62957295707F7627607F762709
:1036B000681B790B80919A03482F55278091180435
:1036C000282F332727FD30958FEF90E0289F80012A
:1036D000299F100D389F100D11248091180890918A
:1036E0001908800F911F2091240830912508821B12
:1036F000930B20916B0430916C04821B930B489FB9
:103700009001499F300D589F300D1124620F731F97
:1037100077FDE4C27595679575956795759567957D
:103720007595679575956795709317046093160462
:103730008091240890912508EC01EE27D7FDE095B3
:10374000FE2F20911E0330911F03409120035091C2
:103750002103DA01C90163E0880F991FAA1FBB1F6B
:103760006A95D1F7821B930BA40BB50BC80FD91F19
:10377000EA1FFB1FCE01DF010496A11DB11DB7FD9D
:10378000A7C243E0B595A795979587954A95D1F738
:1037900080931E0390931F03A0932003B0932103F3
:1037A0008091180890911908800F911F20911E0395
:1037B00030911F034091200350912103821B930BF2
:1037C00090936C0480936B04809124089091250859
:1037D00097FD7CC295958795909325088093240842
:1037E00082E091CE20932D042091780030917900D1
:1037F0008091300490913104280F391F809101018C
:103800008A3009F44DC2220F331F220F331F309329
:10381000310420933004C90137FD51C29595879535
:103820009595879595958795909323048093220489
:103830008091360490913704820F931F97FD44C204
:103840009595879590933704809336042091D804FA
:103850003091D904821B930B90932303809322030E
:103860002091280430912904809122039091230310
:10387000280F391F37FD25C2359527953093290428
:103880002093280483E03FCE20932D0420917800DC
:10389000309179008091320490913304280F391FC0
:1038A000809101018A3009F4F8C1220F331F220FE1
:1038B000331F3093330420933204C90137FDFDC117
:1038C00095958795959587959595879590932504DA
:1038D000809324048091340490913504820F931FC7
:1038E00097FDE9C1959587959093350480933404AD
:1038F0002091DA043091DB04821B930B9093250313
:103900008093240320912A0430912B048091240376
:1039100090912503280F391F37FDCAC1359527958A
:1039200030932B0420932A0481E0EDCD20932D04C5
:1039300080917800909179002091D0043091D10449
:10394000821B930B9093200880931F0880911F087F
:103950009091200820913A0430913B04820F931FEC
:1039600090931D0480931C0482E0CDCD20932D0400
:103970008091CE049091CF0420917800309179000D
:10398000821B930B90931508809314088091140860
:10399000909115082091380430913904820F931FBB
:1039A00090931F0480931E0487E0ADCD20932D04D7
:1039B000809101018A3009F462C1843109F493C114
:1039C000809178009091790020912E0430912F04FD
:1039D000820F931F909321048093200486E093CD5F
:1039E00020932D04809178009091790020913004EB
:1039F00030913104820F931F9093310480933004EF
:103A000010922C0482CD20932D0417CE20932D04E8
:103A10008091780090917900AA2797FDA095BA2F00
:103A2000BC01CD010E94F4647B018C018091C8042B
:103A30009091C904A091CA04B091CB049C01AD013E
:103A4000C801B7010E949464DC01CB01BC01CD0127
:103A50000E94D764DC01CB0190931B0480931A046D
:103A600080911A0490911B0402970CF4BAC08091C3
:103A7000C8049091C904A091CA04B091CB0420E07D
:103A800030E84BE354E4BC01CD010E94FE6488237E
:103A9000DCF58091C8049091C904A091CA04B0914A
:103AA000CB042AE037ED43EA5CE3BC01CD010E9480
:103AB0009564DC01CB018093C8049093C904A09362
:103AC000CA04B093CB0480914B0490914C04845F62
:103AD0009140D0F48091C8049091C904A091CA0487
:103AE000B091CB042DEC3CEC4CEC5DE3BC01CD0182
:103AF0000E949564DC01CB018093C8049093C904B3
:103B0000A093CA04B093CB0481E080931904809100
:103B1000780090917900909317088093160880910F
:103B20001A0490911B04AA2797FDA095BA2F209103
:103B30008A0430918B0440918C0450918D04820F43
:103B4000931FA41FB51F80938A0490938B04A093A6
:103B50008C04B0938D0420918A0430918B044091A1
:103B60008C0450918D0457FD9EC07AE05595479581
:103B7000379527957A95D1F780918A0490918B0497
:103B8000A0918C04B0918D04821B930BA40BB50BF8
:103B900080938A0490938B04A0938C04B0938D043B
:103BA00083E0B1CC20932D048091260390912703CC
:103BB0009C01220F331F280F391F809178009091AC
:103BC000790063E070E00E949965260F371F3695F3
:103BD000279536952795309327032093260385E074
:103BE00092CC80911A0490911B048F5F9F4F0CF030
:103BF0008BCF8091C8049091C904A091CA04B09160
:103C0000CB0420E030E849E054E4BC01CD010E943F
:103C1000016518160CF078CF8091C8049091C90402
:103C2000A091CA04B091CB042AE037ED43EA5CE3EB
:103C3000BC01CD010E949464DC01CB018093C804D7
:103C40009093C904A093CA04B093CB0480914B0411
:103C500090914C04845F914008F056CF8091C80445
:103C60009091C904A091CA04B091CB042DEC3CEC16
:103C70004CEC5DE3BC01CD010E9494643BCF80918C
:103C800078009091790020912E0430912F04820FBA
:103C9000931F0196969587959DCE220F331F09CECF
:103CA000220F331FB4CD21503C4F4F4F5F4F5DCF9C
:103CB0002F5F3F4F33CE019615CE079601CE079664
:103CC000ADCD2F5F3F4FD8CD0196BACD019682CDB5
:103CD000CE01DF010B96A11DB11D53CD615E7F4F5B
:103CE00019CD0196C8CC80917800909179002091EF
:103CF0002E0430912F04820F931F2FEF37E0281BE3
:103D0000390B309321042093200486E0FCCBFF91F3
:103D1000EF91DF91CF91BF91AF919F918F917F9163
:103D20006F915F914F913F912F911F910F91FF9054
:103D3000EF900F900FBE0F901F90189590E2E9E260
:103D4000F3E08FE49193815087FFFCCF08951F9398
:103D500080913D0420912803281710F420933D04FE
:103D600090913C0490FF08C080913D04882309F4A1
:103D7000E6C0815080933D0491FF08C080913D04CE
:103D8000821709F4DBC18F5F80933D04892F992747
:103D900080FF02C081FDD0C00E949E1E90913D0414
:103DA0009A3008F0A2C081E180933E04892F9927C0
:103DB0009F938F938AEE92E09F938F9381E08F93EE
:103DC0000E9456110F900F900F900F900F9020911E
:103DD0003D04822F99278730910509F4B2C18830BC
:103DE00091050CF08CC08330910509F437C2843002
:103DF00091050CF0A7C08130910509F49DC2823075
:103E000091050CF403C310923E048AEA93E09F9359
:103E10008F9311E01F930E94561184E180933E041A
:103E20000F900F900F908091C2049091C304A091C5
:103E3000C404B091C504B7FD22C63AE0B595A79574
:103E4000979587953A95D1F7BF93AF939F938F93AB
:103E500084EB93E09F938F931F930E94561188E207
:103E600080933E048DB79EB707960FB6F8949EBF19
:103E70000FBE8DBF8091BA049091BB04A091BC0489
:103E8000B091BD04B7FDF6C52AE0B595A795979505
:103E900087952A95D1F7BF93AF939F938F9383EC28
:103EA00093E09F938F931F930E9456118CE380930E
:103EB0003E042DB73EB7295F3F4F0FB6F8943EBF83
:103EC0000FBE2DBF80918804909189049F938F939A
:103ED00082ED93E09F938F931F930E9456110F9052
:103EE0000F900F900F900F90ADC780E180933E042C
:103EF000892F99279F938F938FEE92E05DCF8B3020
:103F0000910509F43FC18C3091050CF4CDC08D3082
:103F1000910509F423C58D3091050CF42EC38E3024
:103F2000910509F4B1C50F9709F403C621502093F8
:103F3000280310923D0486C710923D042DCF209394
:103F40003D041ACF8530910509F408C406970CF09A
:103F500091C310923E0480919108E82FFF27EE0F45
:103F6000FF1FE25AF74F808191819F938F93809139
:103F70009008E82FFF27EE0FFF1FE25AF74F8081CE
:103F800091819F938F9381E294E09F938F9311E0AF
:103F90001F930E94561184E180933E048DB79EB713
:103FA00007960FB6F8949EBF0FBE8DBF8091930801
:103FB000E82FFF27EE0FFF1FE25AF74F8081918114
:103FC0009F938F9380919208E82FFF27EE0FFF1F9A
:103FD000E25AF74F808191819F938F9381E394E020
:103FE0009F938F931F930E94561188E280933E0403
:103FF0002DB73EB7295F3F4F0FB6F8943EBF0FBEB7
:104000002DBF80919508E82FFF27EE0FFF1FE25A82
:10401000F74F808191819F938F9380919408E82F2F
:10402000FF27EE0FFF1FE25AF74F808191819F9388
:104030008F9381E494E09F938F931F930E94561176
:104040008CE380933E046DB77EB7695F7F4F0FB6F8
:10405000F8947EBF0FBE6DBF80919708E82FFF27B1
:10406000EE0FFF1FE25AF74F808191819F938F934C
:1040700080919608E82FFF27EE0FFF1FE25AF74FB7
:10408000808191819F938F9381E594E09F938F939B
:104090001F930E9456118DB79EB707960FB6F894DE
:1040A0009EBF0FBE8DBFCEC68930910509F40BC4EB
:1040B0000A970CF01CC210923E0489E695E09F938B
:1040C0008F9311E01F930E94561184E180933E0468
:1040D0000F900F900F9080918404909185049F938E
:1040E0008F9388E795E09F938F931F930E945611BB
:1040F00088E280933E040F900F900F900F900F90E6
:1041000080918804909189049F938F9387E895E02C
:104110009F938F931F930E9456118CE380933E04CC
:104120000F900F900F900F900F90809186049091B8
:1041300087049F938F9386E995E0CCCE10923D043F
:1041400025CE84E180933E0480912603909127033D
:104150009F938F938BE495E09F938F9311E01F9330
:104160000E94561188E280933E040F900F900F90AA
:104170000F900F908091760499279F938F938AE5F3
:1041800095E0A8CE10923E0487E096E09F938F932F
:1041900011E01F930E94561184E180933E040F901A
:1041A0000F900F9080913107992787FD90959F93ED
:1041B0008F9380913007992787FD90959F938F93D8
:1041C00087E196E09F938F931F930E94561188E298
:1041D00080933E048DB79EB707960FB6F8949EBFA6
:1041E0000FBE8DBF80913207992787FD90959F93D1
:1041F0008F938091330799279F938F9387E296E05F
:104200009F938F931F930E9456118CE380933E04DB
:104210002DB73EB7295F3F4F0FB6F8943EBF0FBE94
:104220002DBF8091370799279F938F9380913407F3
:10423000992787FD90959F938F9387E396E09F93AF
:104240008F931F930E9456116DB77EB7695F7F4FA2
:104250000FB6F8947EBF0FBE6DBFF4C510923E043A
:1042600080916208909163089F938F93809160087A
:10427000909161089F938F9381EE93E09F938F932A
:1042800011E01F930E94561184E180933E046DB7A4
:104290007EB7695F7F4F0FB6F8947EBF0FBE6DBFCC
:1042A00080916608909167089F938F93809164082E
:1042B000909165089F938F9381EF93E09F938F93E5
:1042C0001F930E94561188E280933E048DB79EB7DB
:1042D00007960FB6F8949EBF0FBE8DBF80916A08F7
:1042E00090916B089F938F938091680890916908D3
:1042F0009F938F9381E094E09F938F931F930E94ED
:1043000056118CE380933E042DB73EB7295F3F4F93
:104310000FB6F8943EBF0FBE2DBF80916E089091EE
:104320006F089F938F9380916C0890916D089F9375
:104330008F9381E194E083CF8091980880FD1CC029
:1043400084E180933E0485E993E09F938F9311E08D
:104350001F930E94561188E280933E040F900F90A5
:104360000F908CE993E09F938F931F930E945611B7
:104370000F900F900F9066C510923E0480916B04D1
:1043800090916C049F938F9389E593E09F938F9313
:1043900011E01F930E94561184E180933E040F9018
:1043A0000F900F900F900F908091690490916A0484
:1043B0009F938F9388E693E09F938F931F930E9420
:1043C000561188E280933E040F900F900F900F904B
:1043D0000F9080911C0390911D039F938F9387E70B
:1043E00093E09F938F931F930E9456118CE38093C9
:1043F0003E040F900F900F900F900F908091210826
:1044000099279F938F9386E893E064CD892B09F0D9
:104410008DCD10923E0484EF92E09F938F9311E034
:104420001F930E94561184E180933E040F900F90D9
:104430000F9082E690E09F938F938DE090E09F93A2
:104440008F9381E090E09F938F93809101016AE0C8
:104450000E948D65892F99279F938F9380910101E9
:104460000E948D6599279F938F9384E093E09F939B
:104470008F931F930E94561188E280933E042DB7BC
:104480003EB7235F3F4F0FB6F8943EBF0FBE2DBF20
:1044900081E895E09F938F930E944D0499279F9305
:1044A0008F9389E193E09F938F931F930E945611FE
:1044B0008091A7039091A8036DB77EB7695F7F4F86
:1044C0000FB6F8947EBF0FBE6DBF069708F492C476
:1044D00090914104992309F487C48CE380933E04AE
:1044E000892F99279F938F9384E393E0F3CC1092C5
:1044F0003E0485ED95E09F938F9311E01F930E94FA
:10450000561184E180933E040F900F900F9080919C
:10451000900399279F938F938DED95E09F938F93B1
:104520001F930E94561188E280933E040F900F90D3
:104530000F900F900F908091FD039091FE039F9339
:104540008F938BEE95E09F938F931F930E9456114C
:104550008CE380933E040F900F900F900F900F907C
:104560008091B50899279F938F938091B4089927DC
:104570009F938F9389EF95E062CE10923E0487E47B
:1045800096E09F938F9311E01F930E94561184E150
:1045900080933E040F900F900F90809139089927D7
:1045A0009F938F938091380899279F938F93809141
:1045B000370899279F938F938091360899279F9367
:1045C0008F9387E596E09F938F931F930E945611D8
:1045D00088E280933E048DB79EB70B960FB6F89491
:1045E0009EBF0FBE8DBF80913D0899279F938F93EB
:1045F00080913C0899279F938F9380913B0899273E
:104600009F938F9380913A0899279F938F938CE67D
:1046100096E09F938F931F930E9456118CE3809393
:104620003E042DB73EB7255F3F4F0FB6F8943EBF0F
:104630000FBE2DBF8091410899279F938F93809142
:10464000400899279F938F9380913F0899279F93C4
:104650008F9380913E0899279F938F9381E896E0EE
:104660009F938F931F930E9456116DB77EB7655F1E
:104670007F4FEECD10923E0481E195E09F938F93A2
:1046800011E01F930E94561184E180933E040F9025
:104690000F900F908091D0049091D1049F938F93AD
:1046A00080911C0490911D049F938F938EE195E05F
:1046B0009F938F931F930E94561188E280933E042C
:1046C0006DB77EB7695F7F4F0FB6F8947EBF0FBEA0
:1046D0006DBF8091CE049091CF049F938F93809172
:1046E0001E0490911F049F938F938DE295E09F93FA
:1046F0008F931F930E9456118CE380933E048DB7D5
:104700009EB707960FB6F8949EBF0FBE8DBF8091DF
:10471000C8049091C904A091CA04B091CB04BC0113
:10472000CD010E94D764DC01CB019F938F938091D0
:10473000090990910A099F938F938CE395E09F93C9
:104740008F931F930E9456112DB73EB7295F3F4F9D
:104750000FB6F8943EBF0FBE2DBF74C310923E0437
:1047600081E694E09F938F9311E01F930E9456116E
:10477000809101010F900F900F908A3009F4B2C21E
:104780008B3009F4EEC1843109F4EBC18D3009F0AE
:1047900059C384E180933E0480911B0399279F9322
:1047A0008F934091DA045091DB04CA0157FD43C353
:1047B00095958795959587959595879595958795E1
:1047C0009F938F939A0157FD33C335952795359560
:1047D0002795359527958091240490912504821B77
:1047E000930B9F938F9385ED94E09F938F931F93EB
:1047F0000E94561188E280933E046DB77EB7675FD2
:104800007F4F0FB6F8947EBF0FBE6DBF80911A0325
:1048100099279F938F934091D8045091D904CA014E
:1048200057FD0EC395958795959587959595879591
:10483000959587959F938F939A0157FDFEC2359565
:104840002795359527953595279580912204909148
:104850002304821B930B9F938F9389EE94E09F9385
:104860008F931F930E9456118CE380933E048DB763
:104870009EB709960FB6F8949EBF0FBE8DBF80916C
:10488000190399279F938F932091D6043091D704D1
:10489000C90137FDCBC2959587959F938F938091E2
:1048A000200490912104281B390B3F932F938DEF07
:1048B00094E09F938F931F930E9456112DB73EB79C
:1048C000275F3F4F45CF10923E0480917D04909129
:1048D0007E049F938F9385EA95E09F938F9311E0D9
:1048E0001F930E94561184E180933E040F900F9015
:1048F0000F900F900F9080917B0490917C049F9378
:104900008F9381EB95E09F938F931F930E94561195
:1049100088E280933E040F900F900F900F900F90BD
:104920008091790490917A049F938F938DEB95E019
:104930009F938F931F930E9456118CE380933E04A4
:104940000F900F900F900F900F908091770490919F
:1049500078049F938F9389EC95E0BCCA10923E0433
:1049600086E996E09F938F9311E01F930E94561162
:1049700084E180933E040F900F900F908091550832
:1049800099278D969F938F938091540899278D96A0
:104990009F938F938091530899278D969F938F9320
:1049A0008091520899278D969F938F9385EA96E080
:1049B0009F938F931F930E94561188E280933E0429
:1049C0008DB79EB70B960FB6F8949EBF0FBE8DBFE6
:1049D0008091590899278D969F938F9380915808BD
:1049E00099278D969F938F938091570899278D963D
:1049F0009F938F938091560899278D969F938F93BD
:104A000089EB96E09F938F931F930E9456118CE33E
:104A100080933E042DB73EB7255F3F4F0FB6F89405
:104A20003EBF0FBE2DBF80915A0899278D969F9348
:104A30008F938DEC96E09F938F931F930E94561156
:104A40000F900F900F900F900F9080915B0888232C
:104A500009F03AC180915C08882309F027C1809150
:104A60005D08882309F4EEC188E480933E0483EE58
:104A700096E079CC81509C4FAF4FBF4F05CA815013
:104A80009C4FAF4FBF4FD9C910923E0486EE96E0BF
:104A90009F938F9311E01F930E94561184E180939E
:104AA0003E040F900F900F9080916B05E82FFF2729
:104AB000EE0FFF1FEB52FC4F808191819F938F93EC
:104AC00086EF96E09F938F931F930E9456110F904D
:104AD0000F900F900F900F9080916B05811709F048
:104AE000B1C188E280933E0480916D0599279F9320
:104AF0008F9380915D0499279F938F938CE097E02B
:104B00009F938F931F930E9456118CE380933E04D2
:104B10006DB77EB7695F7F4F0FB6F8947EBF0FBE4B
:104B20006DBF80916E0599279F938F9383E297E0E5
:104B3000D1C910923E0488E397E09F938F9311E0D0
:104B40001F930E94561184E180933E040F900F90B2
:104B50000F9080916C0599279F938F9388E497E03D
:104B6000B9C984E180933E044091DA045091DB049A
:104B7000CA0157FD51C19C0135952795359527955B
:104B80003595279535952795C90182959295907F02
:104B90009827807F9827BA01681B790BCB0177FD96
:104BA00039C1959587959F938F933F932F939A0142
:104BB00057FD2DC135952795359527953595279521
:104BC0008091240490912504821B930B9F938F93D3
:104BD00082EA94E09F938F931F930E94561188E27C
:104BE00080933E048DB79EB709960FB6F8949EBF8A
:104BF0000FBE8DBF4091D8045091D904CA0157FD12
:104C000004C19C01359527953595279535952795B0
:104C100035952795C90182959295907F9827807F39
:104C20009827BA01681B790BCB0177FDECC09595ED
:104C300087959F938F933F932F939A0157FDE0C0E1
:104C4000359527953595279535952795809122049B
:104C500090912304821B930B9F938F9384EB94E09A
:104C60009F938F931F930E9456118CE380933E0471
:104C70008DB79EB709960FB6F8949EBF0FBE8DBF35
:104C80002091D6043091D704C90137FDC7C095954E
:104C900087959F938F938091200490912104281BE6
:104CA000390B3F932F9386EC94E049CD84E48093B5
:104CB0003E0480EE96E09F938F931F930E945611BF
:104CC0000F900F900F90CBCE80E480933E048DED3B
:104CD00096E09F938F931F930E9456110F900F9011
:104CE0000F90B8CE84E180933E044091DA04509155
:104CF000DB049A0157FD97C0359527953595279583
:104D000035952795C901880F991F880F991F880F1E
:104D1000991F481B590B5F934F933F932F9380919B
:104D2000240490912504821B930B9F938F938FE60D
:104D300094E09F938F931F930E94561188E2809373
:104D40003E042DB73EB7275F3F4F0FB6F8943EBFE6
:104D50000FBE2DBF4091D8045091D9049A0157FD40
:104D60005FC0359527953595279535952795C901C8
:104D7000880F991F880F991F880F991F481B590B7F
:104D80005F934F933F932F9380912204909123043C
:104D9000821B930B9F938F9381E894E09F938F9353
:104DA0001F930E9456118CE380933E046DB77EB72B
:104DB000675F7F4F0FB6F8947EBF0FBE6DBF8091C7
:104DC000D6049091D7049F938F938091D6049091AD
:104DD000D7042091200430912104821B930B9F93D0
:104DE0008F9383E994E052C98CE380933E0489E475
:104DF00093E0B9CA8CE380933E0487E293E0B3CAA0
:104E0000295F3F4F1DCF019612CF0F96FACE295F33
:104E10003F4FD0CE0196C5CE0F96ADCE019637CF7F
:104E2000295F3F4F9ECF295F3F4F66CF019633CD1D
:104E3000295F3F4FCACC0F96BBCC295F3F4FFFCCB9
:104E40000F96F0CC10923C041F9108951092B90077
:104E50008AE28093B800089585EA8093BC000895A3
:104E600084E98093BC0008951092B9008093BB0040
:104E700085E88093BC0008950E9430271092440476
:104E80008091BB001092430480E88093BC00109294
:104E9000BD001092BA001092BB001092B90010929F
:104EA000B8000E9426270E942C2780E00E94342709
:104EB00008958093BB0085E88093BC00089585EC3D
:104EC0008093BC00089585E88093BC0008951F92EC
:104ED0000F920FB60F9211242F933F934F935F932E
:104EE0006F937F938F939F93AF93BF93EF93FF93B2
:104EF00080914404282F3327442755278F5F8093C0
:104F00004404F90127313105C8F4E05BFF4FEE0F8F
:104F1000FF1F0590F491E02D099480914204E82F41
:104F2000FF27EA5DF74F9091BB0090838F5F8C3035
:104F300008F49DC0109242040E943027109244044D
:104F4000E0C080E80E943427DCC088E90E94342752
:104F5000D8C00E9430278AE090E09093A803809305
:104F6000A7030E942C27CDC084E10E943427C9C02A
:104F700082E10E943427C5C080911B030E94342720
:104F8000C0C080E10E943427BCC080911A030E94F7
:104F90003427B7C0809119030E943427B2C0809192
:104FA0004304E82FFF27E15CF64F8F5F80934304B3
:104FB00080810E943427A5C090914304292FE92FB6
:104FC000FF27EE0FFF1FEE0FFF1FE058FA4F8585FA
:104FD00018160CF054C09C3009F467C0990F892F43
:104FE0008E5A0E9434278DC080914204E82FFF27FB
:104FF000EE5BF74F8091BB0080830E94632781C0E6
:105000008091B900803409F46EC080914204E82F89
:10501000FF27EE5AF74F10828F5F8C3068F11092A5
:1050200042040E94302710924404809145048093EA
:1050300041041092450465C08091B900803309F4A1
:1050400040C00E9430278AE090E09093A8038093AC
:10505000A703109244040E942C2753C00E943027BB
:105060008AE090E09093A8038093A70367CF809392
:1050700042040E94302762CF80934204D2CF9C30FA
:1050800008F0A9CF922F9F5FE92FFF27EE0FFF1F98
:10509000EE0FFF1FE058FA4F858518161CF0292FD8
:1050A0009C3080F39093430496CF1092430483E0A6
:1050B0008093440480914204880F8D5A0E943427C3
:1050C00020C0809145048823C9F4909143049093B3
:1050D0004504E92FFF27EB5CF74F80818F5F09F4D0
:1050E0008FEF8083AECF80914204E82FFF27EE5AE6
:1050F000F74F8C5F80830E945F2797CF9091430486
:10510000E8CF8091BC0080688093BC00FF91EF9154
:10511000BF91AF919F918F917F916F915F914F91CF
:105120003F912F910F900FBE0F901F90189583EC19
:105130008093810080916F00806280936F00109255
:10514000D7041092D6041092D9041092D804109269
:10515000DB041092DA0408951F920F920FB60F929B
:105160001124EF92FF920F931F932F933F934F932E
:105170005F936F937F938F939F93AF93BF93CF93DF
:10518000DF93EF93FF932091860030918700809109
:10519000460490914704281B390B8091860090911A
:1051A00087009093470480934604C9018D5494402E
:1051B000835F9A4178F48091480490914904049760
:1051C00014F010928303C1E0D0E0D0934904C0935F
:1051D0004804A3C0C0914804D0914904CA30D10505
:1051E0000CF09BC0C9018B5F9040845B9140A8F09C
:1051F000FE013196F0934904E0934804E530F1054F
:1052000009F46DC05D98E630F10509F466C05C985C
:10521000379709F460C05B9880C0225D3140FE0181
:10522000EC0FFD1FE25AF74F80819181F901E81BD5
:10523000F90BCF01F7FD6DC0069754F48091760409
:10524000883C08F05FC080917604865F8093760486
:10525000FE01EC0FFD1FE25AF74F80819181AC01F6
:10526000440F551F480F591F420F531F57FD4EC083
:105270007A01F594E794F594E794C90101968E15A7
:105280009F05BCF50894E108F10880917604833C01
:1052900040F18E010C0F1D1FF801E25AF74F80817B
:1052A00091819701281B390BC90163E070E00E94CE
:1052B000AD65CB01880F991F860F971F0C58174FAC
:1052C000F80191838083FE01EC0FFD1FE25AF74F36
:1052D000F182E0828DCF5B9A20C05C9A99CF5D9A73
:1052E00092CFFE01EC0FFD1FEC58F74F1182108298
:1052F000EACF21503040E216F3063CF60894E11C58
:10530000F11CC3CF88EC80937604A2CF4D5F5F4F32
:10531000AFCF909581959F4F8FCFFF91EF91DF9108
:10532000CF91BF91AF919F918F917F916F915F913D
:105330004F913F912F911F910F91FF90EF900F9000
:105340000FBE0F901F90189581E08093900882E027
:105350008093910883E08093920884E0809393087F
:1053600085E08093940886E08093950887E0809399
:10537000960888E08093970808951F9388E68093A5
:1053800098083EE1309399088BEF80939B088AE060
:1053900080939C0830939A0830939E08E4E0E09351
:1053A0009D085FE050939F083093A0081CE0109385
:1053B000A10878E07093A20886EE8093A30830934A
:1053C000A40880E88093A50880E58093A60826E9D4
:1053D0002093A70883E08093A8088EE58093A9080E
:1053E00083E28093AA083093AB081092AC0860E285
:1053F0006093AD081092AE081092AF081092B008FA
:105400001092B1081092C2081092C3081092C408FA
:105410001092C50844E64093B20888E28093B3082E
:105420001092DC0892E39093B4082093B50885E0CD
:105430008093B6089093B7082AE52093B808909314
:10544000B9081092DB082093BA0883E48093BB0864
:105450001092BC0885E58093BD088093BE0880E16A
:105460008093BF086093C0084093C1088FE5809384
:10547000C60883EF8093C8085093C7085093C908A3
:105480008DEF8093CA084093CB082093CC082093DB
:10549000CD082093CE088BE48093CF088093D0086A
:1054A0008093D1081092D20886E08093D30870933D
:1054B000D4082093D5083093D6084093D70840935A
:1054C000D808E093D908A9EAB3E0E1EEF8E00D903E
:1054D00001921A95E1F71F9108951F9388E6809332
:1054E00098085EE1509399088BEF80939B088AE0BF
:1054F00080939C0850939A0850939E0893E0909351
:105500009D081CE010939F0880E18093A00876E03E
:105510007093A10868E06093A20886EE8093A308C8
:105520005093A40880E88093A50880E58093A6089E
:1055300088E78093A7089093A8088EE58093A90830
:1055400083E28093AA085093AB081092AC0830E233
:105550003093AD081092AE081092AF081092B008C8
:105560001092B1081092C2081092C3081092C40899
:105570001092C50844E64093B20888E28093B308CD
:105580001092DC0892E39093B40886E98093B50802
:1055900085E08093B6089093B7082AE52093B80871
:1055A0009093B9081092DB082093BA0883E48093A3
:1055B000BB088CE38093BC0885E58093BD0880938D
:1055C000BE083093BF083093C0089BE49093C10895
:1055D0008FE58093C60883EF8093C80884E18093A9
:1055E000C7088093C9088DEF8093CA084093CB0801
:1055F0002093CC082093CD082093CE089093CF0819
:105600009093D0089093D1081092D2087093D30849
:105610006093D4082093D5085093D6084093D708B8
:105620004093D80884E08093D908A0EBB3E0E1EE82
:10563000F8E00D9001921A95E1F71F91089588EE18
:10564000809398083EE1309399088BEF80939B08F4
:105650008AE080939C0830939A0830939E0893E0E8
:1056600090939D0858E050939F0820E12093A00854
:1056700066E06093A1085093A20886EE8093A30889
:105680003093A40880E88093A50844E64093A608D8
:1056900088E78093A7089093A8088EE58093A908CF
:1056A00083E28093AA0884E18093AB081092AC084F
:1056B0002093AD081092AE081092AF081092B00877
:1056C0001092B1081092C2081092C3081092C40838
:1056D0001092C5084093B20888E28093B3081092F4
:1056E000DC0892E39093B40886E98093B50885E0DE
:1056F0008093B6089093B7082AE52093B808909352
:10570000B9081092DB082093BA0883E48093BB08A1
:1057100086E48093BC0885E58093BD088093BE082D
:1057200080E28093BF088093C0089093C1088FE502
:105730008093C60883EF8093C8083093C7083093DE
:10574000C9088DEF8093CA084093CB082093CC08FA
:105750002093CD082093CE088BE48093CF088093CC
:10576000D0088093D1081092D2086093D308509348
:10577000D4082093D5083093D6084093D708409397
:10578000D80884E08093D9088CE0A8EBB3E0E1EE80
:10579000F8E00D9001928A95E1F70895681779076E
:1057A00044F4680F791F77FD09C0CB019595879563
:1057B0000895681B790B861B970B08956F5F7F4FC9
:1057C000CB019595879508950F931F93CF93C82F7D
:1057D000C150CF3F81F004E610E080916D04882332
:1057E00051F410930204009301048AEF90E00E94A8
:1057F000E314C15090F7CF911F910F9108952F920C
:105800003F924F925F926F927F928F929F92AF9250
:10581000BF92CF92DF92EF92FF920F931F93CF939D
:10582000DF93CDB7DEB7ED970FB6F894DEBF0FBEAE
:10583000CDBF2091D6043091D7048091200490915F
:105840002104281B390B3A87298730934E0920936E
:105850004D0920912A0430912B0437FDD4C735958A
:10586000279535952795359527953AA729A73C87FC
:105870002B877901209128043091290437FDC0C776
:105880003595279535952795359527953CA72BA7D1
:105890003E872D87F0920C09E0920B0930930209A4
:1058A0002093010980913C0990913D09AA2797FD19
:1058B000A095BA2F7C018D01EE0CFF1C001F111F5B
:1058C000E80EF91E0A1F1B1F80911C0490911D04F5
:1058D0009C01442737FD4095542FDA01C901880FF8
:1058E000991FAA1FBB1F880F991FAA1FBB1F820FDA
:1058F000931FA41FB51F820F931FA41FB51FE80E8F
:10590000F91E0A1F1B1F17FD9CC715950795F794D5
:10591000E79415950795F794E794F0923D09E09286
:105920003C098091580990915909AA2797FDA095A3
:10593000BA2F7C018D01EE0CFF1C001F111FE80E19
:10594000F91E0A1F1B1F80911E0490911F049C01C9
:10595000442737FD4095542FDA01C901880F991F5C
:10596000AA1FBB1F880F991FAA1FBB1F820F931F5F
:10597000A41FB51F820F931FA41FB51FE80EF91EA9
:105980000A1F1B1F17FD54C715950795F794E79439
:1059900015950795F794E794F0925909E092580904
:1059A0008091090990910A09AA2797FDA095BA2F1D
:1059B0009C01AD01220F331F441F551F280F391FB3
:1059C0004A1F5B1F80911A0490911B04AA2797FD20
:1059D000A095BA2F280F391F4A1F5B1F57FD16C706
:1059E000559547953795279555954795379527951B
:1059F00030930A092093090920911C0430911D0459
:105A0000C901880F991F880F991F820F931F820F5A
:105A1000931FAA2797FDA095BA2F2091B204309129
:105A2000B3044091B4045091B504820F931FA41F96
:105A3000B51F8093B2049093B304A093B404B093C1
:105A4000B50420911E0430911F04C901880F991FCD
:105A5000880F991F820F931F820F931FAA2797FD0C
:105A6000A095BA2F2091AE043091AF044091B004BC
:105A70005091B104820F931FA41FB51F8093AE04F1
:105A80009093AF04A093B004B093B1048091160931
:105A90009091170920911C0430911D04820F931FCF
:105AA000909317098093160980915009909151099C
:105AB00020911E0430911F04820F931F909351096F
:105AC000809350098091CC049091CD0401969093DD
:105AD000CD048093CC048091AA049091AB04A09152
:105AE000AC04B091AD04BC01CD010E94F4645B0133
:105AF0006C018091160890911708AA2797FDA09530
:105B0000BA2FBC01CD010E94F4647B018C0180910D
:105B1000C8049091C904A091CA04B091CB049C011F
:105B2000AD01C801B7010E949464DC01CB019C0166
:105B3000AD01C601B5010E949564DC01CB01BC0139
:105B4000CD010E94D764DC01CB018093AA0490931D
:105B5000AB04A093AC04B093AD048FEC80937A00B7
:105B60001092180320909A0430909B0440909C045B
:105B700050909D0439E423163BE6330631E043069A
:105B800030E053060CF414C188E49BE6A1E0B0E0D9
:105B90008D839E83AF83B8876090A2047090A30426
:105BA0008090A4049090A50439E463163BE6730644
:105BB00031E0830630E093060CF4DCC488E49BE615
:105BC000A1E0B0E089839A83AB83BC8349855A8581
:105BD000CA01AA2797FDA095BA2F2091920430916F
:105BE00093044091940450919504280F391F4A1F43
:105BF0005B1F2DA33EA34FA358A7A0905409B090BC
:105C00005509C0905609D0905709A80EB91ECA1E52
:105C1000DB1E86017501309164043BA3332309F038
:105C2000DAC080916304882309F0C2C440919808C7
:105C30004CA346FF13C6EBA5FCA5CF01AA2797FDF1
:105C4000A095BA2FBC01CD0129813A814B815C819D
:105C50000E946E659B01AC0197FD2CC7BBE055957A
:105C6000479537952795BA95D1F780918D03E82E02
:105C7000FF2400271127C801B7010E946E6597FD18
:105C800014C7ACE09595879577956795AA95D1F758
:105C90006F87788B898B9A8B6093E4047093E5040B
:105CA0008093E6049093E70429A53AA5C901AA27A1
:105CB00097FDA095BA2FBC01CD012D813E814F816A
:105CC00058850E946E659B01AC0197FD01C7FBE002
:105CD0005595479537952795FA95D1F7C801B7019E
:105CE0000E946E6597FDEFC6DC01CB01ECE0B59537
:105CF000A79597958795EA95D1F78093E8049093B7
:105D0000E904A093EA04B093EB042091E4043091F9
:105D1000E50430938B0820938A082091E8043091A1
:105D2000E90430938F0820938E082F85388949899C
:105D30005A89821B930BA40BB50B8AAF9BAFACAFF8
:105D4000BDAF8093E8049093E904A093EA04B09374
:105D5000EB04A80EB91ECA1EDB1E86017501309128
:105D60008C033DA7332309F0A3C58EA79FA7A8AB3B
:105D7000B9ABB7FD61C62EA53FA548A959A9559550
:105D80004795379527958DA19EA1AFA1B8A5821BF8
:105D9000930BA40BB50B8DA39EA3AFA3B8A78093C1
:105DA000920490939304A0939404B09395048CC5AB
:105DB00098EB291694E939069EEF49069FEF59069C
:105DC0000CF0F1C328EB34E94EEF5FEF2D833E83F7
:105DD0004F835887E1CE2DA13EA14FA158A5209316
:105DE000920430939304409394045093950430911B
:105DF00098083CA310928F0810928E0810928B087E
:105E000010928A081092E0041092E1041092E204C9
:105E10001092E3041092DC041092DD041092DE0470
:105E20001092DF0430918C033DA78091E0049091A3
:105E3000E104A091E204B091E304BC01CD0124E6A9
:105E400030E040E050E00E94E265DA01C901409193
:105E5000DC045091DD04481B590B58A34F8F8091EF
:105E6000DC049091DD04A091DE04B091DF04BC015C
:105E7000CD0124E630E040E050E00E94E265DA0126
:105E8000C9012091E0043091E104821B930B9AA395
:105E900089A38091850390918603A0918703B09197
:105EA0008803BC01CD0128E631E040E050E00E94CB
:105EB0006E65E616F7060807190744F057016801F2
:105EC000A61AB70AC80AD90A8601750117FDA3C424
:105ED000A0925409B0925509C0925609D092570920
:105EE0002BA53CA58F8D98A1280F391F790100277C
:105EF000F7FC0095102F8091960490919704A09143
:105F00009804B0919904E80EF91E0A1F1B1F57014F
:105F100068018091670490916804281B390BC901BE
:105F2000AA2797FDA095BA2F280E391E4A1E5B1E80
:105F300020919D0330919E0340919F035091A003B7
:105F4000221533054405550574F4A8EAEA2EA1E6A6
:105F5000FA2E012D112DE21AF30A040B150B17016D
:105F600028015701680188279927DC01821B930BC0
:105F7000A40BB50B281639064A065B060CF0E9C2DD
:105F8000F8E52F2EFEE93F2EFFEF4F2EFFEF5F2E9D
:105F9000220E331E441E551E20929A0430929B04FA
:105FA00040929C0450929D048201710120929604BB
:105FB00030929704409298045092990429A53AA5EA
:105FC000A9A1BAA12A0F3B1FA901662757FD609519
:105FD000762F80919E0490919F04A091A004B0918F
:105FE000A104480F591F6A1F7B1F5A016B01809142
:105FF000650490916604281B390BC901AA2797FDF7
:10600000A095BA2F680E791E8A1E9B1E8091A1034F
:106010009091A203A091A303B091A4038EAB9FAB78
:10602000A8AFB9AF86159705A805B90564F448EA85
:1060300051E660E070E0481B590B6A0B7B0B3A019C
:106040004B015A016B018EA99FA9A8ADB9ADB095BE
:10605000A095909581959F4FAF4FBF4F68167906D9
:106060008A069B060CF064C2E8E56E2EEEE97E2EF1
:10607000EFEF8E2EEFEF9E2E2EA93FA948AD59AD22
:10608000620E731E841E951E6092A2047092A30479
:106090008092A4049092A504B401A30160929E048E
:1060A00070929F048092A0049092A1048DA19EA161
:1060B000AFA1B8A58093A6049093A704A093A804C9
:1060C000B093A9046092C2047092C3048092C40485
:1060D0009092C5042092BA043092BB044092BC0452
:1060E0005092BD044093BE045093BF046093C0041B
:1060F0007093C104E092B604F092B7040093B80420
:106100001093B904809124039091250397FDA4C3B3
:106110007C01F594E794F594E794F594E794FAA656
:10612000E9A6809122039091230397FD93C38C01EC
:106130001595079515950795159507951CA70BA718
:1061400080912404909125040F9734F458E1E52EB2
:106150005CEFF52EFAA6E9A680912404909125041F
:10616000079734F440E3E42E48EFF42EFAA6E9A6AC
:10617000209101012A3009F46BC28091240490918E
:106180002504815D97400CF007C280912404909112
:106190002504805E974034F080EDE82E87E0F82EED
:1061A000FAA6E9A680912204909123040F9724F483
:1061B00008E11CEF1CA70BA78091220490912304F7
:1061C000079724F400E318EF1CA70BA72A3009F463
:1061D00055C28091220490912304815D974024F060
:1061E00008EE13E01CA70BA78091220490912304D2
:1061F000805E974024F000ED17E01CA70BA7A0914C
:106200009503AA2309F497C0609124037091250394
:106210008091EC049091ED04681B790B209124038C
:1062200030912503280F391F37FD3FC3359527953A
:106230003093ED042093EC04613871050CF43AC2FC
:1062400060E870E07093F3046093F2048A2F99275A
:10625000869FF001879FF00D969FF00D1124CF01CE
:10626000F7FD21C37C01F594E794F594E794F59448
:10627000E794F594E79429A53AA5E20EF31EFAA651
:10628000E9A640912203509123038091EE0490915E
:10629000EF04481B590B2091220330912303280F50
:1062A000391F37FDFDC2359527953093EF042093B4
:1062B000EE04413851050CF4F5C140E850E050932C
:1062C000F1044093F0048A2F9927849FD001859F81
:1062D000B00D949FB00D1124AD019D01B7FDDDC23D
:1062E00089011595079515950795159507951595A8
:1062F0000795EBA5FCA50E0F1F1F1CA70BA7869FDC
:106300009001879F300D969F300D1124C901209177
:10631000240330912503820F931F909325038093CC
:1063200024038091220390912303480F591F509317
:106330002303409322034D855E85141615060CF049
:10634000C1C180918A0890918B0897FDA2C2AA27AB
:1063500097FDA095BA2F6DA5262F332744275527E3
:10636000BC01CD010E946E6597FD8EC2E6E0959559
:10637000879577956795EA95D1F7AF8DB8A1A60F68
:10638000B71FB093FD08A093FC084B855C851416DD
:1063900015060CF0C1C180918E0890918F0897FD71
:1063A0006FC2AA2797FDA095BA2F6DA5262F332778
:1063B00044275527BC01CD010E946E6597FD5BC245
:1063C00046E095958795779567954A95D1F7A9A168
:1063D000BAA1A60FB71FB093F208A093F1083CA191
:1063E00037FDC1C11093F0080093EF08F092FF0849
:1063F000E092FE0880919408E82FFF27EE0FFF1F20
:10640000E25AF74F8081918182599F4FA0917D047C
:10641000B0917E04A817B9070CF0EEC0CD0101962B
:1064200090937E0480937D04DC0180919508E82F91
:10643000FF27EE0FFF1FE25AF74F808191818259AB
:106440009F4F60917B0470917C04681779070CF072
:10645000C4C0CB01019690937C0480937B04BC0163
:1064600080919608E82FFF27EE0FFF1FE25AF74FA3
:106470008081918182599F4F4091790450917A0493
:10648000481759070CF0D5C0CA01019690937A04B9
:1064900080937904AC0180919708E82FFF27EE0FD5
:1064A000FF1FE25AF74F8081918182599F4F2091BF
:1064B000770430917804281739070CF0ABC0C90174
:1064C000019690937804809377049C01B7FD93C163
:1064D000AF3FB10539F034F08FEF90E090937E0438
:1064E00080937D0477FD76C16F3F710539F034F0FC
:1064F0008FEF90E090937C0480937B0457FD70C1F4
:106500004F3F510539F034F08FEF90E090937A04CB
:106510008093790437FD6AC12F3F310509F00CF4EF
:10652000EEC28FEF90E09093780480937704E7C2F7
:106530006092A2047092A3048092A4049092A50495
:10654000A0929E04B0929F04C092A004D092A10495
:10655000ADCD20929A0430929B0440929C045092BC
:106560009D04A0929604B0929704C0929804D09291
:10657000990424CD98EB691694E979069EEF890673
:106580009FEF99062CF528EB34E94EEF5FEF298356
:106590003A834B835C831ACB98EEE92E93E0F92E75
:1065A000FAA6E9A6F2CD2D823E824F825886F4CA21
:1065B0008DA19EA1AFA1B8A580939204909393045E
:1065C000A0939404B0939504909198089CA312CC46
:1065D00069827A828B829C82F9CA808191818259F8
:1065E0009F4F861797070CF03BCF6115710509F493
:1065F00037CFCB0101972FCF8081918182599F4F57
:106600008A179B070CF011CF109709F40ECFCD011C
:10661000019706CF8081918182599F4F82179307FE
:106620000CF054CF2115310509F450CFC901019761
:1066300048CF8081918182599F4F841795070CF034
:106640002ACF4115510509F426CFCA0101971ECF63
:106650008091240490912504835F934034F038EEB8
:10666000E32E33E0F32EFAA6E9A68091240490915C
:1066700025048A5F93400CF495CD8ECD8091220441
:1066800090912304835F934024F008EE13E01CA74D
:106690000BA780912204909123048A5F93400CF40D
:1066A000AECDA9CD3FEF403853070CF008CE40E8FF
:1066B0005FEF05CE8FEF603878070CF0C3CD60E850
:1066C0007FEFC0CD80918A0890918B0897FD9BC188
:1066D000AA2797FDA095BA2FEDA52E2F3327442783
:1066E0005527BC01CD010E946E6597FDADC156E0F6
:1066F00095958795779567955A95D1F72F8D38A100
:10670000261B370B3093FD082093FC084B855C85D6
:10671000141615060CF43FCE80918E0890918F08C8
:1067200097FD6DC1AA2797FDA095BA2FEDA52E2F35
:10673000332744275527BC01CD010E946E6597FD84
:1067400088C136E095958795779567953A95D1F705
:1067500029A13AA1261B370B3093F2082093F108A8
:106760003CA137FF3FCE4BA1442309F03BCE8091A3
:106770006304882309F036CE8B859C85A1E08130A7
:106780009A070CF044C12B853C854FEF203034072D
:106790000CF0A3C189A59AA5280F391F3C872B8728
:1067A00020503F4F3093FF082093FE08AD85BE85F3
:1067B000E1E0A130BE070CF465C12BA53CA5A20FFA
:1067C000B31FBE87AD87A050B140B093F008A0932F
:1067D000EF0810CE10927C0410927B0457FF90CEED
:1067E00010927A041092790437FF96CE10927804B2
:1067F0001092770484C110927E0410927D0472CEB0
:10680000295F3F4F3DC8295F3F4F29C82D5F3F4F4C
:106810004F4F5F4FE5C8E60EF71E081F191FE092A5
:106820005409F0925509009356091093570958CB13
:1068300023E030E040E050E0E20EF31E041F151F9D
:10684000A3C883E090E0A0E0B0E0E80EF91E0A1FC4
:106850001B1F5BC807966BCC07965ACC2DA13EA197
:106860004FA158A52093920430939304409394042D
:1068700050939504BFCA615C7F4F8F4F9F4FA0CD4F
:10688000909581959F4F8DCD615C7F4F8F4F9F4F2E
:106890006DCD909581959F4F5ACD215F3F4F20CD73
:1068A0002F5F3F4F00CD0F96DDCC2F5F3F4FBECC0B
:1068B0002DA13EA14FA158A520939204309393049B
:1068C000409394045093950489859A85AA2797FD4F
:1068D000A095BA2F2AAD3BAD4CAD5DAD820F931F95
:1068E000A41FB51F8B8B9C8BAD8BBE8BBC01CD01C8
:1068F00029813A814B815C810E946E659B01AC01CC
:1069000097FDBBC06BE055954795379527956A95E0
:10691000D1F760918E03862F9927AA27BB278F8BEB
:10692000988FA98FBA8FBC01CD010E946E6597FD2B
:106930009FC02CE095958795779567952A95D1F717
:106940006B8F7C8F8D8F9E8F6093DC047093DD0442
:106950008093DE049093DF046B897C898D899E8906
:106960002D813E814F8158850E946E659B01AC014F
:1069700097FD79C08BE055954795379527958A9572
:10698000D1F76F89788D898D9A8D0E946E6597FDFC
:1069900065C0BCE09595879577956795BA95D1F7D1
:1069A0006AAB7BAB8CAB9DAB6093E0047093E1046E
:1069B0008093E2049093E30429853A8537FD7FC0F4
:1069C000213431050CF431CA6B8D7C8D8D8D9E8DFB
:1069D00097FD2AC0613871058105910564F46AA9A3
:1069E0007BA98CA99DA997FD82C06138710581059D
:1069F00091050CF41ACA81E08093810416CA90951F
:106A000081959F4F8FCE909581959F4F61CEE9A53F
:106A1000FAA58E0F9F1F9C878B8780509140909383
:106A2000FF088093FE08C2CE909580957095619581
:106A30007F4F8F4F9F4FCECF0196A11DB11D8EA7C7
:106A40009FA7A8ABB9AB97C9615C7F4F8F4F9F4F92
:106A50004ECE615C7F4F8F4F9F4F73CE6150704F12
:106A60008F4F9F4F96CF2150384F4F4F5F4F82CF60
:106A70006150704F8F4F9F4F5CCF2150384F4F4F19
:106A80005F4F40CF4D855E856FEF4030560754F520
:106A90008BA59CA5480F591F5E874D8740505F4FBF
:106AA0005093F0084093EF08A5CC6150704F8F4F82
:106AB0009F4FE7C82150384F4F4F5F4FCFC8309599
:106AC00021953F4F7DCF6150704F8F4F9F4F0CC925
:106AD0002150384F4F4F5F4FFAC8F092FF08E092B5
:106AE000FE0864CE1093F0080093EF0883CC9095D5
:106AF0008095709561957F4F8F4F9F4F76CFED9624
:106B00000FB6F894DEBF0FBECDBFDF91CF911F91BE
:106B10000F91FF90EF90DF90CF90BF90AF909F903C
:106B20008F907F906F905F904F903F902F9008953F
:106B3000809101018D3009F455C110927A00809145
:106B40002404909125049093FF088093FE0880917F
:106B50002204909123049093F0088093EF08809191
:106B600020049091210490934E0980934D098091C7
:106B70001C0490911D049C01442737FD4095542F1F
:106B8000DA01C901880F991FAA1FBB1F880F991F1F
:106B9000AA1FBB1F820F931FA41FB51F820F931F35
:106BA000A41FB51F90933D0980933C0980911E045A
:106BB00090911F049C01442737FD4095542FDA0122
:106BC000C901880F991FAA1FBB1F880F991FAA1FF1
:106BD000BB1F820F931FA41FB51F820F931FA41FFB
:106BE000B51F909359098093580980911A04909188
:106BF0001B0490930A09809309098FEC80937A0013
:106C000080919408E82FFF27EE0FFF1FE25AF74FFD
:106C10008081918182599F4FA0917D04B0917E0423
:106C2000A817B9070CF085C0CD01019690937E049A
:106C300080937D04DC0180919508E82FFF27EE0FFB
:106C4000FF1FE25AF74F8081918182599F4F6091D7
:106C50007B0470917C04681779070CF096C0CB0117
:106C6000019690937C0480937B04BC0180919608EC
:106C7000E82FFF27EE0FFF1FE25AF74F8081918127
:106C800082599F4F4091790450917A0448175907CF
:106C90000CF06CC0CA01019690937A048093790439
:106CA000AC0180919708E82FFF27EE0FFF1FE25AF3
:106CB000F74F8081918182599F4F209177043091C5
:106CC0007804281739070CF042C0C9010196909347
:106CD0007804809377049C01B7FD7FC0AF3FB10576
:106CE00011F00CF061C077FD67C06F3F710539F09E
:106CF00034F08FEF90E090937C0480937B0457FDF9
:106D000061C04F3F510539F034F08FEF90E0909320
:106D10007A048093790437FD5BC02F3F310509F079
:106D20000CF463C08FEF90E0909378048093770425
:106D30005CC08081918182599F4F8A179B070CF01C
:106D40007ACF109709F477CFCD0101976FCF80816B
:106D5000918182599F4F821793070CF0BDCF211567
:106D6000310509F4B9CFC9010197B1CF8081918173
:106D700082599F4F841795070CF093CF4115510509
:106D800009F48FCFCA01019787CF80819181825901
:106D90009F4F861797070CF069CF6115710509F4AD
:106DA00065CFCB0101975DCF8FEF90E090937E048C
:106DB00080937D0477FF99CF10927C0410927B041E
:106DC00057FF9FCF10927A041092790437FFA5CF16
:106DD000109278041092770408C010927E041092EA
:106DE0007D0481CF0E947D19A8CE8091BD0899278E
:106DF000AA27BB27BC01CD0124EC39E040E050E0DC
:106E00000E946E65DC01CB018093A1039093A203E5
:106E1000A093A303B093A4038091BE089927AA2747
:106E2000BB27BC01CD010E946E65DC01CB018093C4
:106E30009D0390939E03A0939F03B093A003089596
:106E40006F927F928F929F92AF92BF92CF92DF927A
:106E5000EF92FF920F931F93CF93DF93C0E0D0E0A8
:106E60007E016E011092FF03469AD093D104C09325
:106E7000D004D093CF04C093CE0480E090E0A0E093
:106E8000B0E08093C8049093C904A093CA04B0935F
:106E9000CB04D093DB04C093DA04D093D904C0931D
:106EA000D804D093D704C093D604D0931E09C093BE
:106EB0001D0910928E0310928D03109218040E94E7
:106EC000983584E690E00E94F0140E9498358091F5
:106ED000980880FF10C080911C0390911D03875B70
:106EE000934008F07BC080911C0390911D038E5E3F
:106EF000924008F473C01FE18AE090E00E94F01411
:106F00008091200490912104C80FD91F80912404FE
:106F100090912504E80EF91E80912204909123049B
:106F2000C80ED91E115017FFE7CFA701405F5F4F72
:106F300056954795569547955093DB044093DA0450
:106F40009601205F3F4F36952795369527953093CC
:106F5000D9042093D804CE014096969587959295B2
:106F600082958F7089279F7089279093D70480938B
:106F7000D60490931E0980931D093093D504209365
:106F8000D4045093D3044093D20444E050E0DA0197
:106F90000E94FD65802D853020F1809158099091E7
:106FA000590997FD53C06CE070E00E94AD65709385
:106FB000CF046093CE0480913C0990913D0997FDE8
:106FC00056C06CE070E00E94AD657093D104609390
:106FD000D00480911608909117084DC00E942B197B
:106FE0008ACFDA010E94FD65802D9927982F882786
:106FF000DA0111960E94FD65202D820F911D90935C
:10700000D1048093D004DA0112960E94FD65802D90
:107010009927982F8827DA0113960E94FD65202D65
:10702000820F911D9093CF048093CE04DA011496C1
:107030000E94FD65802D9927982F8827DA011596E3
:107040000E94FD65202D820F911D15C090958195A0
:107050009F4F6CE070E00E94AD657093CF04609329
:10706000CE0480913C0990913D0997FFAACF90955D
:1070700081959F4FA6CFAA2797FDA095BA2FBC0157
:10708000CD010E94F464DC01CB018093C80490938D
:10709000C904A093CA04B093CB041092FF081092C5
:1070A000FE081092F0081092EF0810924E0910920C
:1070B0004D0984E690E00E94F01480911C049091A8
:1070C0001D04AA2797FDA095BA2F9C01AD01220FA0
:1070D000331F441F551F220F331F441F551F280FF6
:1070E000391F4A1F5B1F280F391F4A1F5B1F309330
:1070F0003D0920933C0980911E0490911F04AA270A
:1071000097FDA095BA2F7C018D01EE0CFF1C001F8E
:10711000111FEE0CFF1C001F111FE80EF91E0A1FA5
:107120001B1FE80EF91E0A1F1B1FF0925909E0925F
:1071300058098091A408682E772488249924C901CD
:107140009C01442737FD4095542FC401B3010E9490
:107150006E655B016C016093C2047093C3048093FD
:10716000C4049093C5049701442737FD4095542FDC
:10717000C401B3010E946E65DC01CB018093BA04A7
:107180009093BB04A093BC04B093BD04A0929E0452
:10719000B0929F04C092A004D092A1048093960460
:1071A00090939704A0939804B0939904109292043A
:1071B00010929304109294041092950480911E03EF
:1071C00090911F03A0912003B0912103909319087F
:1071D00080931808109217041092160410928A04D3
:1071E00010928B0410928C0410928D04809188046C
:1071F0009091890490938704809386040E941A5783
:1072000082E390E090930204809301048091BD0892
:107210009927AA27BB27BC01CD0124EC39E040E027
:1072200050E00E946E65DC01CB018856954CAF4F53
:10723000BF4F8093A1039093A203A093A303B093A5
:10724000A4038091BE089927AA27BB27BC01CD01C2
:107250000E946E65DC01CB018856954CAF4FBF4F45
:1072600080939D0390939E03A0939F03B093A003EC
:1072700010928A0310928903809188049091890466
:10728000AA2797FDA095BA2F2091850330918603F8
:107290004091870350918803BC01CD010E946E6527
:1072A000DC01CB018093540990935509A0935609B2
:1072B000B09357091092800410927F0411E010934C
:1072C00000010E94025B80914A04846080934A041A
:1072D0008FEF8093BD091092BE0980E28093BF09B1
:1072E00080919408E82FFF27EE0FFF1FE25AF74F17
:1072F0008081918182599F4F90937E0480937D0479
:1073000080919508E82FFF27EE0FFF1FE25AF74FF5
:107310008081918182599F4F90937C0480937B045C
:1073200080919608E82FFF27EE0FFF1FE25AF74FD4
:107330008081918182599F4F90937A048093790440
:1073400080919708E82FFF27EE0FFF1FE25AF74FB3
:107350008081918182599F4F909378048093770424
:107360001093FF0384E680937604DF91CF911F9101
:107370000F91FF90EF90DF90CF90BF90AF909F90D4
:107380008F907F906F90089580913F0999279093F7
:10739000EB078093EA078091400999279093ED07C6
:1073A0008093EC078091420999279093EF0780938F
:1073B000EE078091410999279093F1078093F00798
:1073C00080916D04882321F08091AE0880FF31C048
:1073D00080914A048C7F80934A0490E010C0A92FCA
:1073E000BB27FD01EB5EF84F8083FD01EB5EF84F9C
:1073F0008081A15CB64F8C939F5F9C3080F480911C
:10740000E003882361F3A92FBB27FD01EB5EF84F52
:107410008081A15CB64F8C939F5F9C3080F38091FC
:10742000E003882359F08091E00381508093E003CA
:1074300005C080914A04816080934A0410924404FC
:10744000109243040E942C27089580919B088B3F43
:1074500068F08B3F09F4B3C28C3F09F431C38D3F10
:1074600009F401C38E3F21F480917704809399033E
:1074700080919A088B3F08F40EC28B3F09F409C231
:107480008C3F09F435C38D3F09F402C38E3F09F4E4
:107490006EC380919A03882309F002C280939A03F5
:1074A00080919C088B3F08F402C28B3F09F4FDC118
:1074B0008C3F09F40BC38D3F09F4EDC28E3F09F4F4
:1074C00053C380919803882309F0F6C180939803F1
:1074D00080919E088B3F68F08B3F09F452C28C3F2D
:1074E00009F4F1C28D3F09F4C1C28E3F21F48091AD
:1074F0007704809397038091A5088B3F68F08B3FBA
:1075000009F45AC28C3F09F4EAC28D3F09F4A8C2BB
:107510008E3F21F480917704809396038091A60892
:107520008B3F08F4D0C18B3F09F4CBC18C3F09F4E9
:10753000EBC28D3F09F4A0C28E3F09F427C38091AE
:1075400094038B3008F4C4C18F3F11F480939403EB
:107550008091A7088B3F68F08B3F09F418C28C3FDD
:1075600009F4CCC28D3F09F48AC28E3F21F4809188
:107570007704809393038091A8088B3F68F08B3F3A
:1075800009F408C28C3F09F4BCC28D3F09F471C2F2
:107590008E3F21F480917704809395032091AD086C
:1075A0002B3F08F499C12B3F09F494C12C3F09F4F7
:1075B000BDC22D3F09F44BC22E3F09F4D2C2209127
:1075C00091038091AE088B3F08F08DC180935E04DB
:1075D0008091AF088B3F68F08B3F09F4E1C18C3F8D
:1075E00009F483C28D3F09F42FC28E3F21F48091AC
:1075F000770480935D048091B0088B3F68F08B3FE7
:1076000009F4D1C18C3F09F46DC28D3F09F43AC22F
:107610008E3F21F48091770480935C048091B108BF
:107620008B3F68F08B3F09F4C1C18C3F09F463C202
:107630008D3F09F42AC28E3F21F480917704809314
:107640005B048091C2088B3F08F45CC18B3F09F456
:10765000B0C18C3F09F42BC28D3F09F41FC28E3F8D
:1076600009F488C290915A048091C3088B3F08F0B6
:1076700051C1482F409359048091C4088B3F68F052
:107680008B3F09F4B7C18C3F09F414C28D3F09F454
:107690000BC28E3F21F4809177048093580480912F
:1076A000C5088B3F68F08B3F09F4A7C18C3F09F4F4
:1076B00010C28D3F09F4CEC18E3F21F48091770432
:1076C000809357048091B2088B3F68F08B3F09F498
:1076D00097C18C3F09F421C28D3F09F4ACC18E3FA4
:1076E00021F480917704809390038091B7088B3FB9
:1076F00068F08B3F09F466C18C3F09F411C28D3FDD
:1077000009F49CC18E3F21F48091770480938F030C
:107710008091BA088B3F68F08B3F09F456C18C3FCB
:1077200009F401C28D3F09F48CC18E3F21F4809190
:10773000770480938E038091BB088B3F68F08B3F6A
:1077400009F446C18C3F09F4E5C18D3F09F470C1CD
:107750008E3F21F48091770480938D038091BC0843
:107760008B3F68F08B3F09F436C18C3F09F4EDC1C3
:107770008D3F09F448C18E3F21F4809177048093B6
:107780008C038091C1088B3F68F08B3F09F426C1C0
:107790008C3F09F4DDC18D3F09F438C18E3F21F4DF
:1077A0008091770480938B038091C7088B3F08F406
:1077B000C2C08B3F09F4BDC08C3F09F4BAC18D3FF4
:1077C00009F427C18E3F09F4DBC18091180982308A
:1077D00008F4B6C08F3F11F4809318099B3F08F45A
:1077E000B1C09B3F09F4FDC09C3F09F490C19D3F8F
:1077F00009F41BC19E3F09F4B1C180910D09882392
:1078000009F0A6C080930D098091C9088B3F08F448
:10781000A6C08B3F09F4A1C08C3F09F493C18D3FF2
:1078200009F4FDC08E3F09F496C180914B09823066
:1078300008F49AC08F3F11F480934B094B3F08F432
:1078400095C04B3F09F4D0C04C3F09F478C14D3F7F
:1078500009F4E8C04E3F09F490C1809111098823D2
:1078600009F08AC0809311098091DA088B3F70F08B
:107870008B3F09F489C08C3F09F45EC18D3F09F448
:10788000CBC08E3F09F085C18091770480935B095E
:1078900080C180917D0480939A03882309F4FECDF2
:1078A000843608F4FDCD84E6F9CD80917D04809383
:1078B0009803882309F40ACE843608F409CE84E6B6
:1078C00005CE80917D04809394038B3008F03CCEEC
:1078D0008AE03CCE20917D04209391038091AE08F4
:1078E0008B3F08F473CE8B3F09F457C08C3F09F4EB
:1078F000F3C08D3F09F4B1C08E3F09F069CE80918D
:10790000770464CE982F90935A048091C3088B3FDC
:1079100008F4AFCE8B3F09F46AC08C3F09F4CDC0A8
:107920008D3F09F4BEC08E3F09F42DC1409159042A
:10793000A3CE80917D0480931809823008F04ACF4D
:1079400081E04ACF892F80930D09882309F45ACF0B
:107950008A3F08F459CF8AEF55CF80917D048093F8
:107960004B09823008F066CF81E066CF842F809388
:107970001109882309F476CF8A3F08F475CF8AEF7E
:1079800071CF80917D04B5CD80917D047FCF8091B2
:107990007D04EFCD80917D04FFCD80917D0416CED6
:1079A00080917D0426CE80917D0436CE80917D0429
:1079B00046CE90917D04A7CF80917D04ADCD80917E
:1079C0007D0454CD80917D04A1CE80917D04B1CE03
:1079D00080917D04C1CE80917D04D1CE80917D04C3
:1079E000E1CE80917D04AFCF80917D04C0CF4091E6
:1079F0007D0440CE80917D0450CE80917D0460CE88
:107A000080917D0470CE80917904B9CE8091790403
:107A1000C9CE809179048FCF8091790437CF80913E
:107A200079049DCF80917904A2CF809179048BCF86
:107A30008091790491CE8091790455CE809179041A
:107A400065CE8091790475CE80917904D2CD209154
:107A5000790442CF8091790433CE80917904B6CDF8
:107A60008091790459CD8091790400CD8091790479
:107A700040CD8091790490CD8091790424CF80917C
:107A8000790477CD80917904C7CD80917904D7CDE1
:107A90008091790400CF8091790409CF9091790485
:107AA00032CF40917904E6CD80917904F6CD909162
:107AB0007B0429CF80917B04F0CD40917B04DACD0B
:107AC00080917B04D3CC80917B0413CD80917B0487
:107AD000EECE80917B04F4CD80917B0477CD8091B4
:107AE0007B041ACD80917B0497CD80917B0481CD5E
:107AF00080917B04D0CE80917B04A1CD80917B04CA
:107B000038CD80917B0448CD80917B04DCCE809180
:107B10007B0419CF80917B041FCE80917B04E3CD41
:107B200080917B04F3CD80917B0403CE20917B0474
:107B3000D3CE80917B04FFCE80917B04A7CE809131
:107B40007B0415CF80917B040ACF80917B0417CEF4
:107B500080917B0427CE8091770401CF80917704B8
:107B6000F2CE20917704B8CE80917704A0CE809198
:107B7000770491CE90917704C6CE80917704F7CEAA
:107B800080917704D8CE4091770474CD80917704AA
:107B90009ACE33272F5F3F4F8CE398E2B9010E94C2
:107BA000AD6570939C0360939B038091A3088093C1
:107BB0004C098091A2088093030908952F923F9267
:107BC0004F925F926F927F928F929F92AF92BF92ED
:107BD000CF92DF92EF92FF920F931F93CF93DF9399
:107BE000CDB7DEB7EA970FB6F894DEBF0FBECDBFB4
:107BF0000E94FF2B209101012C3010F00C949E4626
:107C0000299AA0906E04B0906F04BA82A9828091E4
:107C10007604843610F00C94AB4680910E038823D2
:107C200011F40C94A84880911005909111050097CB
:107C300011F40C94C44A0197909311058093100598
:107C40002A3011F40C94CC4A243111F40C94CC4A0F
:107C5000289880914B0490914C04895E934010F4D5
:107C60000C94C04A8091AA08282F33273A8329838D
:107C700081E08093830480919008A82FBB27AA0FEE
:107C8000BB1FFD01EC58F74F1182108280919108C3
:107C9000282F3327220F331FC9018C58974FFC011F
:107CA00011821082A25AB74F11961C921E92225A2C
:107CB000374FD90111961C921E9280919308E82F9C
:107CC000FF27EE0FFF1FE25AF74F118210828091BB
:107CD0008303815080938303809183038F3F29F036
:107CE000A0918304AA2309F4D5C20E94253A809169
:107CF0009008E82FFF27EE0FFF1FE25AF74F808111
:107D000091814C01AA2497FCA094BA2C80919108EF
:107D1000E82FFF27EE0FFF1FE25AF74F8081918176
:107D20006C01EE24D7FCE094FE2C8091C50880FF06
:107D300077C0F094E094D094C094C11CD11CE11C95
:107D4000F11CC501B4012FE93BE140E050E00E9485
:107D50006E654B015C01C701B6010E946E656B0147
:107D60007C01D501C4018C199D09AE09BF09BC0174
:107D7000CD0120E137E240E050E00E94E265890158
:107D8000C80CD91CEA1CFB1CC701B60120E137E274
:107D900040E050E00E94E265DA01C9014801AA24EE
:107DA00097FCA094BA2C909581959F4F6C01EE247E
:107DB000D7FCE094FE2C1EE781169104A104B104C7
:107DC00014F00C94CF4A23E882162FEF92062FEF7F
:107DD000A2062FEFB20644F4A3E88A2EAFEF9A2E44
:107DE000AFEFAA2EAFEFBA2E3EE7C316D104E104DF
:107DF000F1042CF0FDE7CF2ED12CE12CF12C43E83F
:107E0000C4164FEFD4064FEFE4064FEFF40644F4E8
:107E1000E3E8CE2EEFEFDE2EEFEFEE2EEFEFFE2EAD
:107E200080911F0590912005AA2797FDA095BA2F54
:107E300095018401081B190B2A0B3B0BC901B801E2
:107E400023E030E040E050E00E94E265DA01C90141
:107E5000880F991FAA1FBB1F820F931FA41FB51F56
:107E60008C018091210590912205AA2797FDA0956C
:107E7000BA2FA7019601281B390B4A0B5B0BCA01CD
:107E8000B90123E030E040E050E00E94E265DA0111
:107E9000C901880F991FAA1FBB1F820F931FA41F20
:107EA000B51FFC019092200580921F05D0922205FB
:107EB000C092210580912305909124059C01220FF9
:107EC000331F280F391F80919F08682F7727689DDF
:107ED000C001699D900D789D900D1124280F391FC8
:107EE00037FF02C00C943A53359527953595279561
:107EF0008091A008482F5527409FC001419F900DB9
:107F0000509F900D1124820F931F9093240580930E
:107F1000230520914B0530914C05821B930B9093C8
:107F200075048093740480912505909126059C0129
:107F3000220F331F280F391F6C9DC0016D9D900DBE
:107F40007C9D900D1124280F391F37FF02C00C941F
:107F5000365335952795359527954E9FC0014F9FF0
:107F6000900D5E9F900D1124820F931F9093260514
:107F7000809325052091490530914A05821B930B7A
:107F8000909373048093720480919308E82FFF27E5
:107F9000EE0FFF1FE25AF74F8081918190958195F6
:107FA0009F4F8330910514F40C945E4A029790938E
:107FB0007104809370040E944D608C018091940341
:107FC0009927AA2797FDA095BA2FBC01CD010E9441
:107FD000F464DC01CB0120E030E040E251E4BC017C
:107FE000CD010E949564DC01CB01BC01CD010E9452
:107FF000D764DC01CB018093520960919303809395
:10800000F60860930E098091370780FF06C08091C3
:108010005B09813810F00C94F44A10936F040093BC
:108020006E0480916E0490916F0497FF02C00C94CF
:1080300030538091980882FD02C00C94A74A109298
:108040001F094091740450917504CA0157FF02C082
:108050000C94B24A959587959595879597FF02C0A0
:108060000C94BB4A20914F043091500428173907D3
:1080700014F00C94664ACA0157FF02C00C943254A3
:1080800097FF02C00C942F54BC01759567957595A8
:1080900067956536710514F40C94694A64E670E0DE
:1080A0004091720450917304CA0157FD02C00C94B0
:1080B000724A0396959587959595879597FD02C089
:1080C0000C947A4A909581959F4F20914D04309160
:1080D0004E042817390714F40C94834AC9010197F8
:1080E000A0918304AA2311F40C949D4A1092500489
:1080F00010924F0410924E0410924D04509191082A
:10810000E52FFF27EE0FFF1FE25AF74F4091B80807
:10811000242F3327808191812817390734F48091E7
:10812000DB0882FF02C00C94EF4AE52FFF27EE0F19
:10813000FF1FE25AF74F842F99272091B908821B1D
:108140009109208131812817390714F410926204B3
:10815000E52FFF27EE0FFF1FE25AF74F842F9927D5
:1081600022273327281B390B80819181821793079F
:1081700034F48091DB0883FF02C00C94EA4A8091BA
:108180006104882391F0E52FFF27EE0FFF1FE25ACD
:10819000F74F8091B9089927841B9109208131817B
:1081A0008217930714F40C94764B60919008E62F95
:1081B000FF27EE0FFF1FE25AF74F242F332780814E
:1081C00091812817390734F48091DB0880FF02C0C1
:1081D0000C94E44A50915F04552399F0E62FFF2751
:1081E000EE0FFF1FE25AF74F842F99272091B9080D
:1081F000821B9109208131812817390714F40C94CE
:10820000714BE62FFF27EE0FFF1FE25AF74F842F27
:10821000992722273327281B390B808191818217C8
:10822000930734F48091DB0881FF02C00C94DF4A8D
:1082300080916004882391F0E62FFF27EE0FFF1F47
:10824000E25AF74F8091B9089927841B9109208140
:1082500031818217930714F40C947A4B8091620455
:10826000882331F480916104882311F40C94DC4A52
:1082700091E0552331F480916004882311F40C942B
:10828000574B81E08093640410926304109262045F
:1082900010926104F0916304FF8FFF2321F4809119
:1082A0006404882369F08091B7089927A980BA806F
:1082B0008A159B0514F49A83898381E08093810455
:1082C000AA2311F40C94594A10927104109270046C
:1082D0001092750410927404109273041092720438
:1082E0009AE59093520988E780931F099093F608C6
:1082F0008C8B80930E0910926304109264041F8E7D
:1083000020911209309113094091140950911509D7
:10831000C090C204D090C304E090C404F090C5049F
:10832000C88AD98AEA8AFB8A2C0D3D1D4E1D5F1D25
:108330008091190990911A09A0911B09B0911C090B
:10834000E090BA04F090BB040091BC041091BD040D
:10835000EF8AF88E098F1A8F8E0D9F1DA01FB11FF7
:10836000A0900509B0900609C0900709D0900809AF
:10837000ADA6BEA6CFA6D8AAC090BE04D090BF041A
:10838000E090C004F090C104CB8EDC8EED8EFE8EAA
:10839000EDA4FEA40FA518A9AB8CBC8CCD8CDE8CF3
:1083A000EA0CFB1C0C1D1D1DEDA6FEA60FA718ABAD
:1083B000C090F708D090F808E090F908F090FA081B
:1083C000C9A6DAA6EBA6FCA6E090B604F090B70426
:1083D0000091B8041091B904EDA2FEA20FA318A752
:1083E000A9A4BAA4CBA4DCA4AE0CBF1CC01ED11E91
:1083F000A9A6BAA6CBA6DCA6B0906404BD8ABB2011
:1084000011F00C94F5490F8D002311F00C94F549EF
:108410008093190990931A09A0931B09B0931C0922
:1084200020931209309313094093140950931509AE
:108430008091160890911708815092400CF09FC6C9
:1084400080916D04882309F09AC68091140490915C
:1084500015048F3F910509F008F4A0C7ED89EE23BC
:1084600011F00C94834BFF8DFF2311F00C94834B80
:10847000009181040F87002311F00C94834B10911D
:10848000C0081CA3112311F40C94834B2DA53EA509
:108490004FA558A920930509309306094093070971
:1084A0005093080989A59AA5ABA5BCA58093F708A8
:1084B0009093F808A093F908B093FA0880911209F4
:1084C00090911309A0911409B0911509B7FF02C04A
:1084D0000C941956292E3A2E4B2E552447FC5A94AB
:1084E00020921209309213094092140950921509F2
:1084F0008091190990911A09A0911B09B0911C094A
:10850000B7FF02C00C941356892F9A2FAB2FBB27AD
:10851000A7FDBA958B839C83AD83BE838093190995
:1085200090931A09A0931B09B0931C098091A40889
:10853000E82EFF24002711272091B2043091B304C4
:108540004091B4045091B504C801B7010E946E6512
:1085500097FF02C00C943156672E782E892E9924ED
:1085600087FC9A942091AE043091AF044091B004FE
:108570005091B104C801B7010E946E6597FF02C017
:108580000C942B56A72EB82EC92EDD24C7FCDA94E6
:10859000D201C10186199709A809B9092091BF081C
:1085A000E22EFF2400271127BC01CD01A80197016D
:1085B0000E94E26539014A0119012A018B819C81DF
:1085C000AD81BE818A199B09AC09BD09BC01CD01F1
:1085D000A80197010E94E265D401C30197FE02C081
:1085E0000C942556892F9A2FAB2FBB27A7FDBA9540
:1085F000BC01DA01C90157FF02C00C941F56892F34
:108600009A2FAB2FBB27A7FDBA956C0180914F0421
:108610009091500481349105D4F480914D0490914F
:108620004E04813491059CF480919308E82FFF2734
:10863000EE0FFF1FE25AF74F808191810190F08188
:10864000E02DF7FF02C00C949C567A9734F080918D
:10865000BD098F3F11F40C94B455EB8CFC8C0D8D3F
:108660001E8D288939894A895B89E21AF30A040B2D
:10867000150BEFAAF8AE09AF1AAFE0920005F09221
:10868000010500930205109303058DA19EA1AFA1E2
:10869000B8A5EF88F88C098D1A8D8E199F09A00B4B
:1086A000B10B8F839887A987BA878093040590932D
:1086B0000505A0930605B09307050FA918AD29ADD0
:1086C0003AAD009308051093090520930A053093ED
:1086D0000B0580930C0590930D05A0930E05B093A8
:1086E0000F0580919E0490919F04A091A004B091E9
:1086F000A104801B910BA20BB30B80939E0490935B
:108700009F04A093A004B093A1048091960490913B
:108710009704A0919804B09199042F8138854985D8
:108720005A85821B930BA40BB50B809396049093F0
:108730009704A0939804B09399043CA1332371F15A
:1087400020917F04309180042138310594F080918C
:10875000D6049091D70401969093D7048093D604C1
:1087600080911D0990911E09019690931E09809396
:108770001D0920583F4F94F48091D6049091D7045E
:1087800001979093D7048093D60480911D0990910E
:108790001E09019790931E0980931D091092800471
:1087A00010927F0401E0A02EB12C8FA998ADA9AD45
:1087B000BAADB7FF02C00C94FD5581509240A04065
:1087C000B0401CF014E0A12EB12C80912D059091A9
:1087D0002E05A0912F05B0913005E0901209F09080
:1087E000130900911409109115098E199F09A00B06
:1087F000B10B815E914BAF4FBF4F8F539C49A0404F
:10880000B04010F40C946B55F091BE09FE8BF93119
:1088100014F40C94E755B0922805A09227058FA96F
:1088200098ADA9ADBAAD81509041A040B04014F4CC
:108830000C94745580912905882311F40C944956A1
:1088400070936604609365048FA998ADA9ADBAAD25
:10885000B7FF02C00C94E0569C01AD01B7FF02C007
:108860000C94EF56B9E05595479537952795BA95ED
:10887000D1F78091270590912805820F931F90933F
:108880002805809327052FA938AD49AD5AAD57FF6C
:1088900002C00C94E95639014A01A3E095948794EB
:1088A00077946794AA95D1F713012401F9E86F161C
:1088B000F3E17F06F0E08F06F0E09F0644F0F8E871
:1088C0006F2EF3E17F2E812C912C13012401D40112
:1088D000C30197FE02C00C94B056892F9A2FAB2F7C
:1088E000BB27A7FDBA95680F791F2FA938AD49ADF1
:1088F0005AAD203080EF38078FEF48078FEF5807C9
:1089000014F00C94885580912A05882311F40C9456
:1089100006567093660460936504DA01C90157FF37
:1089200002C00C9493569C01AD01B7FF02C00C9499
:10893000CB5669E055954795379527956A95D1F7B8
:108940008091270590912805820F931F9093280509
:10895000809327052FA938AD49AD5AAD57FF02C006
:108960000C94C55639014A0143E095948794779455
:1089700067944A95D1F798E769169CEE79069FEFC0
:1089800089069FEF990644F438E7632E3CEE732E78
:108990003FEF832E3FEF932E6092170570921805DC
:1089A0008092190590921A05D401C30197FE02C066
:1089B0000C94AA56892F9A2FAB2FBB27A7FDBA95E7
:1089C0006091650470916604680F791FACA12A2F2D
:1089D000332780912705909128052817390724F41B
:1089E0003093280520932705BE89BB2379F02B2FD0
:1089F000332727FD3095809127059091280528176A
:108A0000390724F430932805209327052FA938AD82
:108A100049AD5AAD213831054105510574F08091B9
:108A2000DA049091DB042091270530912805820F0C
:108A3000931F9093DB048093DA048FA998ADA9ADBE
:108A4000BAAD80589F4FAF4FBF4F74F48091DA0496
:108A50009091DB042091270530912805821B930B10
:108A60009093DB048093DA04B1E0AB2EB12C8F81BC
:108A70009885A985BA85B7FF02C00C944E568150DF
:108A80009240A040B0401CF0A4E0AA2EB12C20E0FF
:108A900030E040E050E08091310590913205A091A6
:108AA0003305B09134056090190970901A098090CF
:108AB0001B0990901C0986199709A809B909815EBC
:108AC000914BAF4FBF4F8F539C49A040B04028F00F
:108AD000FE89F93114F40C94D155B0922805A09276
:108AE00027058F819885A985BA8581509041A0403E
:108AF000B04014F40C947C5580912B05882311F41C
:108B00000C943C56D0926804C09267048F8198857B
:108B1000A985BA85B7FF02C00C94D756B7FF02C02B
:108B20000C947E56F9E0B595A79597958795FA959B
:108B3000D1F7A80EB91EB0922805A09227052F8163
:108B4000388549855A8557FF02C00C947856E3E072
:108B50005595479537952795EA95D1F72938F3E14B
:108B60003F07F0E04F07F0E05F0714F40C946856FD
:108B700088E893E1A0E0B0E080931B0590931C058A
:108B8000A0931D05B0931E0580911B0590911C05B7
:108B9000A0911D05B0911E05B7FF02C00C9472563E
:108BA000892F9A2FAB2FBB27A7FDBA95C0906704DA
:108BB000D0906804C80ED91E2F81388549855A8502
:108BC000203080EF38078FEF48078FEF580714F0F9
:108BD0000C94785580912C05882311F40C94375609
:108BE000D0926804C0926704DA01C90157FF02C03D
:108BF0000C948A569C01AD01B7FF02C00C948456B8
:108C0000B9E05595479537952795BA95D1F7809155
:108C1000270590912805820F931F90932805809334
:108C200027052F81388549855A8557FF02C00C9446
:108C3000A456A3E05595479537952795AA95D1F762
:108C400028379CEE39079FEF49079FEF590714F02B
:108C50000C945E5688E79CEEAFEFBFEF80931B0548
:108C600090931C05A0931D05B0931E0580911B05D4
:108C700090911C05A0911D05B0911E05B7FF02C083
:108C80000C94B656892F9A2FAB2FBB27A7FDBA9508
:108C9000C0906704D0906804C80ED91EACA12A2FDA
:108CA000332780912705909128052817390724F448
:108CB0003093280520932705BE89BB2379F02B2FFD
:108CC000332727FD30958091270590912805281797
:108CD000390724F430932805209327052F81388500
:108CE00049855A85213831054105510574F0809137
:108CF000D8049091D9042091270530912805820F3E
:108D0000931F9093D9048093D8048F819885A98567
:108D1000BA8580589F4FAF4FBF4F0CF00AC5809166
:108D2000D8049091D9042091270530912805821B01
:108D3000930B9093D9048093D804FBC42998A090F6
:108D40006E04B0906F04BA82A98280917604843652
:108D500010F40C940D3E809176048D3810F40C9430
:108D6000673E109283049091AB0882E3989FC00104
:108D700011249093110580931005E981FA81B99728
:108D80000CF09BC480914B0490914C048F3F910553
:108D900019F010F00C9429531092F4041092F50479
:108DA0001092F6041092F7041092F8041092F9044D
:108DB0001092FA041092FB048A3F910511F40C946E
:108DC0003F5530919208E32FFF27EE0FFF1FE25A25
:108DD000F74F80819181813591050CF4E9C0409174
:108DE0006D04442309F0E4C080919308E82FFF2725
:108DF000EE0FFF1FE25AF74F808191818C3491056D
:108E000014F40C948D54809112058F5F893C10F4FA
:108E10000C9463552C3010F00C94CE552998109278
:108E20006D041092120510924C0410924B04609144
:108E30009008E62FFF27EE0FFF1FE25AF74F8081C1
:108E400091818734910514F00C94CA555091910882
:108E5000E52FFF27EE0FFF1FE25AF74F8081918128
:108E60000190F081E02DF7FF02C00C94BC56E7346E
:108E7000F1050CF470C021E0A52FBB27AA0FBB1F82
:108E8000A25AB74F8D919C9111978734910544F068
:108E9000E62FFF27EE0FFF1FE25AF74F80819181E7
:108EA0008D919C918734910564F0E62FFF27EE0F9A
:108EB000FF1FE25AF74F80819181873491050CF0B2
:108EC00022E0E52FFF27EE0FFF1FE25AF74F8081C8
:108ED00091818634910564F4E62FFF27EE0FFF1F82
:108EE000E25AF74F80819181873491050CF023E09D
:108EF000E52FFF27EE0FFF1FE25AF74F8081918188
:108F00008A5B9F4F64F4E62FFF27EE0FFF1FE25AA4
:108F1000F74F80819181873491050CF024E0E52F93
:108F2000FF27EE0FFF1FE25AF74F808191818A5B86
:108F30009F4F64F4E62FFF27EE0FFF1FE25AF74F13
:108F400080819181863491050CF425E0822F0E9466
:108F5000120450919108E52FFF27EE0FFF1FE25AF0
:108F6000F74F808191810190F081E02DF7FF02C0E1
:108F70000C9457567E9714F00C9494558091900859
:108F8000E82FFF27EE0FFF1FE25AF74F80819181F4
:108F90008A5B9F4F14F00C94945581E080932B07CB
:108FA00088EE93E09093020480930104309192083C
:108FB000E32FFF27EE0FFF1FE25AF74F80819181C9
:108FC0008B5A9F4F14F00C94673ED0909308ED2D70
:108FD000FF27EE0FFF1FE25AF74F80819181855BDB
:108FE0009F4F14F00C940954809113058F5F893CB6
:108FF00010F40C942E5588EC8093130581E090E0DA
:1090000090934C0480934B0481E080936D04109204
:10901000FC041092FD041092FE041092FF041092C2
:10902000920410929304109294041092950410925A
:109030008E0410928F0410929004109291048091EB
:10904000A408E82EFF240027112780913C09909165
:109050003D099C01442737FD4095542FC801B701B5
:109060000E946E65DC01CB018093A2049093A3045F
:10907000A093A404B093A504809158099091590934
:109080009C01442737FD4095542FC801B7010E9429
:109090006E65DC01CB0180939A0490939B04A093AE
:1090A0009C04B0939D048091C2049091C304A0914C
:1090B000C404B091C50480939E0490939F04A09330
:1090C000A004B093A1048091BA049091BB04A09134
:1090D000BC04B091BD048093960490939704A09330
:1090E0009804B09399041092F4041092F50410922D
:1090F000F6041092F7041092F8041092F9041092FA
:10910000FA041092FB0480914A04886080934A0418
:109110008091C50881FD02C00C940B548091980881
:1091200080FF10C080911C0390911D03875B9340CA
:1091300038F480911C0390911D038E5E924010F4D0
:109140000E942B190E942037D09093080C940B5446
:1091500080911103909112038F5F9F4F11F00C9437
:10916000133E88E99AE3909302048093010480E01F
:109170009CE090931203809311030C94133E909003
:10918000BD096FEF961611F40C9440538091A4081A
:10919000A82EBB24CC24DD24688979898A899B89FF
:1091A000A60195010E94E26579018A0180913C093E
:1091B00090913D09AA2797FDA095BA2FE81AF90AC0
:1091C0000A0B1B0B6F89788D898D9A8DA6019501ED
:1091D0000E94E26559016A018091580990915909EC
:1091E000AA2797FDA095BA2FA81AB90ACA0ADB0ABE
:1091F000292C332427FC3094432C532CC201B10179
:10920000A80197010E946E6597FD78C23B014C0151
:10921000F9E09594879477946794FA95D1F7C20111
:10922000B101A60195010E946E6597FF02C00C94E2
:109230006B545B016C01E9E0D594C794B794A79493
:10924000EA95D1F780914F049091500481349105B3
:109250003CF480914D0490914E0481349105C4F00A
:10926000D401C30197FE02C00C943A553C014D0154
:109270009594879477946794D601C501D7FE02C070
:109280000C9435555C016D01D594C794B794A7949F
:1092900080919308E82FFF27EE0FFF1FE25AF74F48
:1092A000808191810190F081E02DF7FF02C00C9444
:1092B00066547A97A4F0C401B30123E030E040E0A3
:1092C00050E00E94E26539014A01C601B50123E080
:1092D00030E040E050E00E94E26559016A0180916F
:1092E000BF09282F332727FD3095432F532F2615ED
:1092F00037054805590514F439014A01992787FDB6
:109300009095909581959F4FAA2797FDA095BA2F8C
:10931000681679068A069B0614F43C014D012A154D
:109320003B054C055D0514F459016A01A816B90600
:10933000CA06DB0614F45C016D018091A2049091D1
:10934000A304A091A404B091A50486199709A809C3
:10935000B9098093A2049093A304A093A404B093AA
:10936000A50480919A0490919B04A0919C04B091D3
:109370009D048A199B09AC09BD0980939A049093B6
:109380009B04A0939C04B0939D048091140490913D
:1093900015048F3F910511F008F060C8ADA4BEA47C
:1093A000CFA4D8A8A0920509B0920609C0920709D7
:1093B000D0920809C9A4DAA4EBA4FCA4C092F708CF
:1093C000D092F808E092F908F092FA08009181042E
:1093D0000F87A0907004B0907104C501B7FE09C258
:1093E000882799278A199B0904C21092B204109207
:1093F000B3041092B4041092B5041092AE0410920B
:10940000AF041092B0041092B1041092120910929D
:10941000130910921409109215091092190910924B
:109420001A0910921B0910921C0919A61AA61BA64C
:109430001CA620E030E040E050E02DA73EA74FA75B
:1094400058AB8091A2049091A304A091A404B09180
:10945000A50480939E0490939F04A093A004B093CE
:10946000A10480919A0490919B04A0919C04B091D6
:109470009D048093960490939704A0939804B093CE
:10948000990410921504109214041092660410921C
:10949000650410926804109267043D89332311F02B
:1094A0000C9425424F8D442311F00C9425420C94CA
:1094B0001842B0900E09BC8A0C9480413FEF8E3F59
:1094C00093070CF073C002960C94D73FB90161501A
:1094D00070404091720450917304CA0157FF02C05A
:1094E0000C945940959587959595879597FF02C05F
:1094F0000C94624020914D0430914E042817390796
:1095000014F00C946E40CA0157FF02C00C943A54F8
:1095100097FF02C00C94375495958795959587953C
:109520008536910514F40C94704084E690E0A09187
:109530008304AA2311F00C94764090934E048093F8
:109540004D047093500460934F040C947E406093DC
:109550001F094091740450917504CA0157FD02C05F
:109560000C942A400396959587959595879597FD38
:1095700002C00C943240909581959F4F0C943240DC
:1095800010926D040C94673E10926D041092830447
:109590002A3011F00C94243E289A0C94293EBDE701
:1095A0008B2E912CA12CB12C0C94E33E10927104C3
:1095B000109270040C94DB3F982F0C94394181E099
:1095C000809360040C942E4181E080935F04582FB7
:1095D0000C94014181E0809361040C94D54081E0BA
:1095E000809362040C94A84080913007282F332781
:1095F00027FD309580919F08482F5527249FC00153
:10960000259F900D349F900D11242091740430916A
:109610007504820F931F9093750480937404809156
:109620003107992787FD9095849FD001859FB00DC4
:10963000949FB00D1124CD012091720430917304D8
:10964000820F931F9093730480937204809132076A
:10965000992787FD90952091700430917104820FB5
:10966000931F909371048093700480913407282F86
:10967000332727FD309580919D089927289FF00179
:10968000299FF00D389FF00D1124F0938A03E09389
:1096900089038091330799278017910714F00C9460
:1096A0000D4090936F0480936E040C94114090933E
:1096B0006304809364040C944A4180916D04882370
:1096C00009F460CB80914B0490914C04FFEF8F3FE5
:1096D0009F0709F45BCB019690934C0480934B0455
:1096E00055CB10925F0450E00C940141109261043C
:1096F0000C94D540109260040C942E4161507E4F22
:109700008F4F9F4F83CD60E070E06B01109281041A
:109710001F86E0901209F09013090091140910912E
:1097200015096090190970901A0980901B09909092
:109730001C0980911F09882309F031C71092680421
:10974000109267041092660410926504E0922D0551
:10975000F0922E0500932F0510933005609231058D
:109760007092320580923305909234051092B204C3
:109770001092B3041092B4041092B5041092AE0487
:109780001092AF041092B0041092B1041092AA0487
:109790001092AB041092AC041092AD041092120916
:1097A00010921309109214091092150910921909B8
:1097B00010921A0910921B0910921C0910920509A7
:1097C0001092060910920709109208091092F708E2
:1097D0001092F8081092F9081092FA0810921504E5
:1097E00010921404A0907004B0907104C501B7FCED
:1097F000F7CD40977CF068EE262E63E0362E30924F
:10980000A6032092A5038091980884FD03C081E0FF
:1098100080931605D090A108ED2CFF240027112776
:10982000B501882777FD8095982F9501B7FC0CC767
:10983000442737FD4095542F0E946E659B01AC0173
:10984000C801B7010E946E6597FDF9C659E095956C
:109850008795779567955A95D1F79B018D2D992717
:109860008A9DA0018B9D500D9A9D500D1124CA0117
:1098700057FDE3C69595879595958795280F391FD0
:10988000C901AA2797FDA095BA2F8093FC04909355
:10989000FD04A093FE04B093FF0420919204309144
:1098A00093044091940450919504281B390B4A0B62
:1098B0005B0B213563EC360760E0460760E0560736
:1098C0000CF464C680E593ECA0E0B0E080939204D1
:1098D00090939304A0939404B09395048091920480
:1098E00090919304A0919404B0919504805B9C4363
:1098F000AF4FBF4F64F480EB9CE3AFEFBFEF8093BB
:10990000920490939304A0939404B0939504609070
:109910008804709089046114710409F446C580912B
:10992000980883FF42C588899989AA89BB89B7FDB0
:10993000ADC709E0B595A795979587950A95D1F795
:1099400098AF8FAB97FDACC78F89988DA98DBA8DD5
:10995000B7FDA1C719E0B595A795979587951A9575
:10996000D1F7BC0197FDAEC7CFA8D8ACC616D706B5
:1099700014F478AF6FAB6FA978AD77FDA0C72B015A
:109980005594479455944794559447940894411C92
:10999000511CACE1EA2EA2E0FA2E6E0C7F1C730182
:1099A0000027F7FC0095102F24EE3DEF620E731E8A
:1099B000A0905409B0905509C0905609D09057090D
:1099C0008091850390918603A0918703B0918803CD
:1099D00088A399A3AAA3BBA3C601B50128A139A155
:1099E0004AA15BA10E94E265E21AF30A040B150B7F
:1099F000C801B70128E631E040E050E00E94E2658E
:109A0000DC01CB018C01045B104080904D099090EB
:109A10004E09C40197FC4EC78138910514F000E04F
:109A200010E02090A5033090A6032114310499F48E
:109A3000AFA9B8AD59977CF480917F0490918004D0
:109A4000800F911F9093800480937F04809116056E
:109A5000882309F0EAC7C801880F991F880F991F4A
:109A6000880F991FB2010E94AD659B01442737FD05
:109A70004095542F2A0D3B1D4C1D5D1D209354090C
:109A8000309355094093560950935709F090960327
:109A90006F2D7727EFA9F8AD6E9FC0016F9F900DD6
:109AA0007E9F900D112497FD03C7959587959595F9
:109AB0008795959587959595879595958795681B35
:109AC000790B78AF6FAB77FDDAC62114310409F05A
:109AD00008C700914F041091500480914D0490915B
:109AE0004E04080F191F17FDE3C715950795159527
:109AF000079515950795005C1F4FCA01B90128A16C
:109B000039A14AA15BA10E94E265DA01C901209155
:109B1000860430918704442737FD4095542F821BDB
:109B2000930BA40BB50B845E9D4FAF4FBF4FBC0191
:109B3000CD0128E631E040E050E00E94E265DC0122
:109B4000CB01845B9040CFA8D8AC8C9D50018D9DFB
:109B5000B00C9C9DB00C1124C501B8010E94AD65EC
:109B600083E0F89E8001112418AF0FAB061717078A
:109B70000CF0BFC6B801CB01AA2797FDA095BA2F5C
:109B80002091920430919304409194045091950453
:109B9000820F931FA41FB51F809392049093930488
:109BA000A0939404B09395048091150581508F3F44
:109BB00009F404C4809315051F85112381F01092C8
:109BC000F8041092F9041092FA041092FB04109217
:109BD000F4041092F5041092F6041092F7042D8903
:109BE000222309F0C4C480911F099927AA27BB2703
:109BF000BC01CD01288939894A895B890E946E653B
:109C0000DC01CB01BC01CD0128EF3AE240E050E09D
:109C10000E94E26529013F8D332309F0A5C480919C
:109C20001F099927AA27BB27BC01CD012F89388D91
:109C3000498D5A8D0E946E65DC01CB01BC01CD01BE
:109C400028EF3AE240E050E00E94E2651901A0905E
:109C5000F108B090F20849ECA416B1040CF479C4F0
:109C6000E8ECAE2EB12CB092F208A092F10800916F
:109C7000FC081091FD08093C11050CF462C408ECC5
:109C800010E01093FD080093FC088091FE0890916D
:109C9000FF08AA2797FDA095BA2F20915209C22E3E
:109CA000DD24EE24FF24BC01CD01A70196010E9412
:109CB0006E659B01AC01C501AA2797FDA095BA2F3F
:109CC00067E0880F991FAA1FBB1F6A95D1F7280F5D
:109CD000391F4A1F5B1F57FD70C486E05595479595
:109CE000379527958A95D1F7C201820F931F98AFB8
:109CF0008FAB3C018091EF089091F008AA2797FD67
:109D0000A095BA2FBC01CD01A70196010E946E65F6
:109D10009B01AC01C801AA2797FDA095BA2F07E0C7
:109D2000880F991FAA1FBB1F0A95D1F7280F391F4B
:109D30004A1F5B1F57FD3CC416E055954795379564
:109D400027951A95D1F75101A20EB31E6501880C13
:109D5000991CC401AA2797FDA095BA2F2091F60857
:109D6000332744275527BC01CD010E946E657B0136
:109D70008C0197FD40C4B6E015950795F794E794DC
:109D8000BA95D1F73C89832F9927AA27BB27209121
:109D9000A6043091A7044091A8045091A904BC01E5
:109DA000CD010E946E65DC01CB01BC01CD0120EF2D
:109DB00035E540E050E00E94E2654701820E931EC7
:109DC000A40194018FA998AD815090442CF0E0E05B
:109DD000F0E4F8AFEFAB3F01F0E06F16F0EC7F0678
:109DE0000CF0A8C380E090EC9093FF088093FE08ED
:109DF00001E0C01600E4D00624F0A12CA0E4BA2EA5
:109E0000650110E0C11610ECD1060CF08EC380E0A5
:109E100090EC9093F0088093EF08415050441CF070
:109E200020E030E4490180E0881680EC98060CF0D0
:109E300077C380E090EC90934E0980934D09809118
:109E400041048823C1F080914B0490914C04029707
:109E5000C09788F4A981BA811A161B0664F481E0C0
:109E600090E090934C0480934B0480910309E82F79
:109E7000FF27FA83E983A980BA80AA0CBB1CAA0C2D
:109E8000BB1CBA82A9820E941D5FA81AB90ABA82B5
:109E9000A982A0904C098A2D9927880F991F880FB5
:109EA000991F80559040C980DA808C159D0514F467
:109EB0009A838983E980FA80F092E107E092E007D3
:109EC0008091FC049091FD04A091FE04B091FF04E8
:109ED000880F991FAA1FBB1F880F991FAA1FBB1F9E
:109EE00000914D0910914E09081B190B1EAB0DABCB
:109EF0009701213A31050CF42CC2C701F7FCBEC30F
:109F0000959587954DA95EA98417950714F49EAB86
:109F10008DAB909581959F4FADA9BEA9A817B907A4
:109F20000CF428C22A2D3327220F331F220F331F90
:109F3000C901A981BA818A1B9B0BEDA9FEA98E17C5
:109F40009F0714F49EAB8DAB69817A81621B730B02
:109F5000CDA8DEA8C616D70614F47EAB6DAB009173
:109F6000FE081091FF088091740490917504081BFD
:109F7000190B1093100900930F0990901F09992055
:109F800009F4F8C2481A590AC201AA2797FDA095F8
:109F9000BA2F2091F4043091F5044091F6045091C9
:109FA000F704820F931FA41FB51F8093F4049093AE
:109FB000F504A093F604B093F7046091F404709153
:109FC000F5048091F6049091F70461302AEF72074E
:109FD00020E0820720E0920774F080E09AEFA0E092
:109FE000B0E08093F4049093F504A093F604B0934A
:109FF000F704BC01CD01603036E073073FEF830703
:10A000003FEF930774F480E096E0AFEFBFEF8093EB
:10A01000F4049093F504A093F604B093F704BC0104
:10A02000CD01E0909B03F0909C039701442737FDFE
:10A030004095542F0E94E2656801C20ED31EB09075
:10A040008B036B2D7727882799272DA93EA937FDEC
:10A05000F0C237FDD9C23595279549815A81240F21
:10A06000351F442737FD4095542F0E946E6597FD9C
:10A07000DBC226E095958795779567952A95D1F768
:10A080009B016C157D050CF46B0166277727621B1D
:10A09000730BC616D7060CF46B010091EF081091F4
:10A0A000F0088091720490917304081B190B1093AF
:10A0B000EE080093ED08992009F462C2281A390AC3
:10A0C000C101AA2797FDA095BA2F2091F8043091DD
:10A0D000F9044091FA045091FB04820F931FA41FCE
:10A0E000B51F8093F8049093F904A093FA04B093F9
:10A0F000FB046091F8047091F9048091FA04909146
:10A10000FB0461305AEF750750E0850750E0950772
:10A1100074F080E09AEFA0E0B0E08093F8049093B0
:10A12000F904A093FA04B093FB04BC01CD016030A4
:10A13000A6E07A07AFEF8A07AFEF9A0774F480E0E2
:10A1400096E0AFEFBFEF8093F8049093F904A093EB
:10A15000FA04B093FB04BC01CD019701442737FDFD
:10A160004095542F0E94E2657801E20EF31E6B2D9C
:10A170007727882799272DA93EA937FD38C237FDB3
:10A1800021C235952795E981FA812E0F3F1F44277B
:10A1900037FD4095542F0E946E6597FD23C216E04F
:10A1A00095958795779567951A95D1F79B016E15CB
:10A1B0007F050CF47B0166277727621B730BE6167D
:10A1C000F7060CF47B018601222717FD2095322F1C
:10A1D0000B871C872D873E8780910309282F332703
:10A1E0003AAB29AB4A2D55275CAB4BABBFE3CB2E2B
:10A1F000B9E0DB2E00E815E02701662457FC6094E7
:10A20000762C8DA99EA94C01AA2497FCA094BA2C67
:10A21000ABE03A2EF0E2EF2EF9E0FF2E06C0F8AFE9
:10A22000EFABEFA9D601EC93E0C5F8012585121636
:10A230000CF0A3C049815A81CA01AA2797FDA095B5
:10A24000BA2F332727FD3095432F532FBC01CD0163
:10A250000E946E6597FDA2C0E6E09595879577957B
:10A260006795EA95D1F778AF6FABF8018685282F0F
:10A27000332727FD3095432F532F6B857C858D85A4
:10A280009E850E946E6597FD84C056E095958795E2
:10A29000779567955A95D1F72FA938AD260F371FB7
:10A2A00038AF2FABF8018785282F332727FD30954E
:10A2B000432F532FC301B2010E946E6597FD64C006
:10A2C00046E095958795779567954A95D1F72FA99B
:10A2D00038AD260F371F38AF2FABF8018089282FF4
:10A2E000332727FD3095432F532FC501B4010E941A
:10A2F0006E65DC01CB01B7FD43C036E0B595A7958F
:10A30000979587953A95D1F7F701608171812FA9CB
:10A3100038AD820F931F0E94CE2BD7018D939C9353
:10A3200097FD41C0959587959595879598AF8FAB8B
:10A33000E9A9FAA98E179F070CF471CF2BA93CA9A4
:10A340004FA958AD241735070CF06BCF38AF2FABA2
:10A3500068CFEDA9FEA9E135F10524F000E510E094
:10A360001EAB0DAB2DA93EA9205B3F4F0CF0DACD03
:10A3700080EB9FEF9EAB8DABD5CDD6011C9235C542
:10A38000CF96A11DB11DB9CF615C7F4F8F4F9F4FFD
:10A3900097CF615C7F4F8F4F9F4F77CF615C7F4F2F
:10A3A0008F4F9F4F59CF0396BDCF80904D0990900E
:10A3B0004E0980911505815008F0FCCB88E180930F
:10A3C00015058091A4089927880F991F880F991F58
:10A3D0007C010027F7FC0095102F688979898A890C
:10A3E0009B89A80197010E94E2653093D3072093CF
:10A3F000D2076F89788D898D9A8DA80197010E9467
:10A40000E2653093D5072093D40780913C09909161
:10A410003D0997FD22C295958795959587959093CF
:10A42000D7078093D607809158099091590997FDD5
:10A4300012C295958795959587959093D9078093A6
:10A44000D8079092DB078092DA0780916B04909195
:10A450006C049093DD078093DC078091160890913F
:10A4600017089093DF078093DE077092E3076092EE
:10A47000E20780912603909127039093E50780934C
:10A48000E4078091540990915509A0915609B09123
:10A49000570920918503309186034091870350919D
:10A4A0008803BC01CD010E94E2653093E907209347
:10A4B000E8078091760499279093E7078093E60751
:10A4C00080912B0799279093F9078093F807809143
:10A4D000FD039091FE039093FB078093FA07809110
:10A4E000BE09992787FD90959093090880930808E5
:10A4F0008091C009992790930D0880930C08809152
:10A500004B0590914C0590930F0880930E08809115
:10A51000490590914A0590931108809310084CCBFF
:10A5200030934E0920934D098ACCB092F008A09246
:10A53000EF0873CCEFA8F8ACF092FF08E092FE08A9
:10A5400057CC6FEF083316070CF09FCB08E31FEFD3
:10A5500098CB58E3A5165FEFB5060CF088CB78E3EF
:10A56000A72E7FEFB72E7FCB2224332470CB442439
:10A57000552451CBC801AA2797FDA095BA2F09CD24
:10A58000C801AA2797FDA095BA2F9FCD20939204CA
:10A590003093930440939404509395049FC9D092B0
:10A5A0006804C09267047093660460936504CEC823
:10A5B000215C3F4F4F4F5F4FBFCB215C3F4F4F4F11
:10A5C0005F4F8BCB2F5F3F4F35952795E981FA8100
:10A5D0002E0F3F1F442737FD4095542F0E946E6574
:10A5E00097FFDDCD615C7F4F8F4F9F4FD8CD30956A
:10A5F00021953F4FC4CD2FE330E040E050E0E20E24
:10A60000F31E041F151FB7CB2F5F3F4F35952795BE
:10A6100049815A81240F351F442737FD4095542F17
:10A620000E946E6597FF25CD615C7F4F8F4F9F4FD6
:10A6300020CD309521953F4F0CCD03961BC961501D
:10A640007E4F8F4F9F4F02C9222733272A193B097C
:10A65000EFC880914A04826080934A040C94E146DA
:10A6600010926F0410926E040C9419402D5F3F4FAE
:10A670000C94A93F2D5F3F4F0C94743F019640CC42
:10A680008091A408E82EFF24002711276889798982
:10A690008A899B89A80197010E94E26539014A01D4
:10A6A00080913C0990913D09AA2797FDA095BA2F6A
:10A6B000681A790A8A0A9B0A6F89788D898D9A8D22
:10A6C000A80197010E94E26559016A018091580929
:10A6D00090915909AA2797FDA095BA2FA81AB90AEF
:10A6E000CA0ADB0AD401C30197FCE9C13C014D0150
:10A6F00054E095948794779467945A95D1F7D6014E
:10A70000C501D7FCD8C15C016D0144E0D594C79464
:10A71000B794A7944A95D1F780914F049091500433
:10A72000813491050CF4F0C0C401B30123E030E0A2
:10A7300040E050E00E94E26539014A01C601B501DE
:10A7400023E030E040E050E00E94E26559016A01F8
:10A7500080919308E82FFF27EE0FFF1FE25AF74F73
:10A76000808191810190F081E02DF7FD9DC17A9764
:10A77000A4F0C401B30123E030E040E050E00E94C7
:10A78000E26539014A01C601B50123E030E040E04D
:10A7900050E00E94E26559016A0181E26816710485
:10A7A000810491042CF030E2632E712C812C912CC9
:10A7B00090EE69169FEF79069FEF89069FEF990645
:10A7C00044F420EE622E2FEF722E2FEF822E2FEF09
:10A7D000922EA1E2AA16B104C104D1042CF090E299
:10A7E000A92EB12CC12CD12CB0EEAB16BFEFBB06FD
:10A7F000BFEFCB06BFEFDB0614F00C949D4980EE53
:10A80000A82E8FEFB82E8FEFC82E8FEFD82E0C9476
:10A810009D4910921305ED2DFF27EE0FFF1FE25A01
:10A82000F74F808191818C3491058CF080911405D3
:10A830008F5F893C08F415C110926D0488EC8093F9
:10A84000140510924C0410924B040C94673E109225
:10A8500014050C94673E0396ECCD0396DCCD03966D
:10A860000C944440909581959F4F0C9440400396E2
:10A870000C948C4A909581959F4F0C94884A84EF54
:10A8800091E09093A6038093A5038EC981509E4FBB
:10A89000AF4FBF4F4EC881509E4FAF4FBF4F5AC8AA
:10A8A0005C01B094A194B108B394B8AEAFAA4CC8FF
:10A8B0004F96FBC88827992788199909ADC8695F01
:10A8C0007F4F5DC8709561957F4F4EC8F095E195BB
:10A8D000FF4F0C94594961507E4F8F4F9F4F0C94FE
:10A8E00019490894210831083092A6032092A50343
:10A8F0005BC98FA998AD909581959F4F681779078F
:10A900000CF039C9BC0137C980914D0490914E04B7
:10A91000813491050CF41CCF07CF80819181855B38
:10A920009F4F0CF0D4C0809112058F5F8093120569
:10A93000893C10F40C94D8472C3008F0BDC12998FC
:10A94000A4E0B0E08FEF082E0E940A6610926D041A
:10A950001092120510924C0410924B040E94203762
:10A96000A4E0B0E08091D0049091D10497FD1CC286
:10A97000892F990F990B082E0E940A66A5E0B0E076
:10A980008091D0049091D104082E0E940A66A6E01E
:10A99000B0E08091CE049091CF0497FD02C2892F40
:10A9A000990F990B082E0E940A66A7E0B0E08091EB
:10A9B000CE049091CF04082E0E940A6608E010E0B1
:10A9C0008091C8049091C904A091CA04B091CB04AD
:10A9D000BC01CD010E94D764DC01CB019C0197FD35
:10A9E000B0C1832F992787FD9A95D801082E0E9420
:10A9F0000A6609E010E08091C8049091C904A09112
:10AA0000CA04B091CB04BC01CD010E94D764DC0123
:10AA1000CB01D801082E0E940A660E944D040E94B4
:10AA2000E42B309192080C94D847C301AA2797FDD4
:10AA3000A095BA2FBC01CD0128A139A14AA15BA1E3
:10AA40000E946E655B016C010E94E2653093870491
:10AA500020938604109216050C942B4D80931305B9
:10AA6000DACE809314050C94673E0196A11DB11DAA
:10AA70000C9442490196A11DB11D0C94364981E008
:10AA8000809316051092FC041092FD041092FE04AF
:10AA90001092FF0410929204109293041092940466
:10AAA000109295040C94E146F095E195FF4F5FCE2E
:10AAB000095F1F4F1AC80F96A11DB11D24CE0F9616
:10AAC000A11DB11D13CE809312050C94D84740935D
:10AAD00012050C94D847B0922805A0922705209122
:10AAE000BE092E8B0C940F44109229050C947544CA
:10AAF00010922C050C944E4620931B0530931C0598
:10AB000040931D0550931E0510922B050C94DC45B7
:10AB100020921705309218054092190550921A0597
:10AB200010922A050C94E6440E944D044DE560E91C
:10AB300078E00E94F7038091980880FF10C0809110
:10AB40001C0390911D03875B934038F480911C0394
:10AB500090911D038E5E924010F40E942B190E946A
:10AB600020370E94F00359CF709366046093650408
:10AB7000D0926804C0926704CB0177FD04C1BC0188
:10AB800075956795C601D7FCFCC06C01D594C79438
:10AB90000C942D43509191080C943B47299A0C94A6
:10ABA0000F4720931B0530931C0540931D055093C0
:10ABB0001E051092280510922705E8EE2E2EE3E0E0
:10ABC0003E2E3092A6032092A5030C944E4660922E
:10ABD0001705709218058092190590921A05109227
:10ABE00028051092270588EE282E83E0382E309213
:10ABF000A6032092A5030C94E644B095A0959095E9
:10AC000081959F4FAF4FBF4F0C94DD4320921705A6
:10AC1000309218054092190550921A0581E08093F0
:10AC20002A050C94E64481509F4FAF4FBF4F0C94C0
:10AC3000844281509F4FAF4FBF4F0C946A42815066
:10AC40009F4FAF4FBF4F0C94FF4281509F4FAF4F6C
:10AC5000BF4F0C94F24261507F4F8F4F9F4F0C9427
:10AC6000C24261507F4F8F4F9F4F0C94AC4281E0A6
:10AC700080932C050C944E4620931B0530931C05A5
:10AC800040931D0550931E0581E080932B050C9485
:10AC9000DC4581E0809329050C947544B095A0951E
:10ACA000909581959F4FAF4FBF4F0C943F45F095C6
:10ACB000E195FF4F0C94BA47299A42CE20931B0589
:10ACC00030931C0540931D0550931E050C94364689
:10ACD00020931B0530931C0540931D0550931E05C2
:10ACE0000C94C44581509F4FAF4FBF4F0C94D0453B
:10ACF000295F3F4F4F4F5F4F0C94A74581509E4FA8
:10AD0000AF4FBF4F0C94924521503E4F4F4F5F4F76
:10AD10000C940046B095A095909581959F4FAF4FAC
:10AD2000BF4F0C94FA45B095A095909581959F4F93
:10AD3000AF4FBF4F0C949344F095E195FF4F0C94A7
:10AD4000254321503F4F4DCE295F3F4F4F4F5F4F1F
:10AD50000C94194681509F4FAF4FBF4F0C94DA446B
:10AD600081509F4FAF4FBF4F0C946D4481509F4F08
:10AD7000AF4FBF4F0C944246F095E195FF4F0C94B6
:10AD80003747019602CF0196FACE295F3F4F4F4FCA
:10AD90005F4F0C94B24421503E4F4F4F5F4F0C9485
:10ADA000994481509F4FFBCD81509F4FE1CDB0958D
:10ADB000A095909581959F4FAF4FBF4F0C948E45B6
:10ADC000B095A095909581959F4FAF4FBF4F0C9434
:10ADD0002C44295F3F4F4F4F5F4F0C944B44215001
:10ADE0003E4F4F4F5F4F0C9432443A94E2E0F0E014
:10ADF000EE0EFF1E0C5F1F4F0894C11CD11C37FEC6
:10AE000014CAEA960FB6F894DEBF0FBECDBFDF912D
:10AE1000CF911F910F91FF90EF90DF90CF90BF9057
:10AE2000AF909F908F907F906F905F904F903F90EA
:10AE30002F9008958091410590914205A09143057E
:10AE4000B09144058093390590933A05A0933B0552
:10AE5000B0933C0580913D0590913E05A0913F0542
:10AE6000B09140058093350590933605A093370542
:10AE7000B0933805089510924C0510924B0510922E
:10AE80004A0510924905089584B1806A84B93D9AB3
:10AE900082E58CBD1DBC459A91E090935E098AEADB
:10AEA0008093620983E8809363098AE08093640950
:10AEB000109266091092650910926809109267094C
:10AEC0001092C00910928409909385098DE08093B7
:10AED00086099093870986E0809388090895EF9208
:10AEE000FF920F931F93F8948091A4089927880FDD
:10AEF000991F880F991F7C010027F7FC0095102FE0
:10AF00008091C2049091C304A091C404B091C5047F
:10AF1000BC01CD01A80197010E94E265309366094A
:10AF2000209365098091BA049091BB04A091BC0460
:10AF3000B091BD04BC01CD01A80197010E94E2655A
:10AF4000309368092093670920915409309155097D
:10AF50004091560950915709DA01C90173E0880FF1
:10AF6000991FAA1FBB1F7A95D1F7820F931FA41FA9
:10AF7000B51F820F931FA41FB51F20918503309129
:10AF800086034091870350918803BC01CD010E9444
:10AF9000E26530936E0920936D09E091CC04F09145
:10AFA000CD048091160990911709BF010E94AD65EB
:10AFB000CB019B01220F331F220F331F280F391F94
:10AFC000280F391F37FDF2C0359527953595279500
:10AFD00030936A0920936909809150099091510931
:10AFE000BF010E94AD659B01220F331F220F331F4B
:10AFF000260F371F260F371F37FDD5C035952795EC
:10B000003595279530936C0920936B091092CD04E8
:10B010001092CC041092170910921609109251093F
:10B02000109250098091640999278C30910509F498
:10B030008AC08D3091050CF06AC08A30910509F400
:10B0400033C10B9709F4B5C07894809184098823A3
:10B0500009F4A0C020918A0930918B09C90181505F
:10B060009E4F8F5F9340C8F440918C0950918D0999
:10B07000CA0181509E4F8F5F934078F48091980869
:10B0800085FF0BC030934C0520934B0550934A0528
:10B09000409349058AEF80934E05809190099091E5
:10B0A000910921E0893692070CF0E8C09C01909349
:10B0B0008904809388048091860490918704281BDA
:10B0C000390BC901845E9D4F68E671E00E94AD6551
:10B0D000845B90409093850480938404209194092C
:10B0E0003091950980910104909102048217930791
:10B0F00040F480912B07882321F43093020420939D
:10B10000010480918909873609F055C1BCC08D3092
:10B11000910509F404C10E9709F096CF8091850935
:10B1200080937509809186098093760980918709BB
:10B130008093770980918809809378098091010133
:10B140008093790981CF80912B07863018F0109277
:10B150002B0785E08093750980916B0490916C04B6
:10B1600090937809809377098091D9088093760924
:10B170008091CF08809379098091D00880937A09D3
:10B180008091D10880937B097894809184098823E9
:10B1900009F060CF10924C0510924B0510924A05B1
:10B1A0001092490508C12D5F3F4F28CF2D5F3F4FBB
:10B1B0000BCF80919208E82FFF27EE0FFF1FE25A76
:10B1C000F74F0190F081E02DE038F1050CF0D8C088
:10B1D0002FEFE138F20714F4E1E8FFEFE09375098F
:10B1E00080919308E82FFF27EE0FFF1FE25AF74FD9
:10B1F0000190F081E02DE038F1050CF4D4C0EFE7C8
:10B20000F0E0E093760980919108E82FFF27EE0F98
:10B21000FF1FE25AF74F0190F081E02DE038F10571
:10B220000CF4B9C0EFE7F0E0E09377098091900863
:10B23000E82FFF27EE0FFF1FE25AF74F0190F08132
:10B24000E02DE038F1050CF49EC0EFE7F0E0E0936C
:10B25000780980917D048093790980917B048093A3
:10B260007A098091790480937B0980917704809397
:10B270007C098091760480937D09E6CE2091880434
:10B280003091890418CF809196098093BD098091EF
:10B2900097098093BF09809198098093BE09809196
:10B2A00099098093C00987C080915E0480937509D5
:10B2B00080915D048093760980915C048093770986
:10B2C00080915B048093780980915A048093790976
:10B2D0008091590480937A098091580480937B0966
:10B2E0008091570480937C0980914A0480937D0962
:10B2F00080914A04837F80934A0480912603909131
:10B30000270380937E098091A90880937F09A2E09A
:10B31000B0E00E94FD65802D8093800995CE8091DC
:10B32000CA08809375098091CB0880937609809133
:10B33000CC08809377098091CD088093780980911B
:10B34000CE08809379098091D20880937A09809100
:10B35000D30880937B098091D40880937C098091E5
:10B36000D70880937D098091D50880937E098091CC
:10B37000D60880937F098091D8088093800964CE95
:10B38000EFE7F0E02BCF8FEFE138F8070CF05FCF5D
:10B39000E1E8FFEF5CCF6FEFE138F6070CF044CF48
:10B3A000E1E8FFEF41CF4FEFE138F4070CF029CF90
:10B3B000E1E8FFEF26CF1F910F91FF90EF900895E6
:10B3C00080915E09882309F43BC0459882E699E0A4
:10B3D0009093600980935F0980914D05E82FFF27C6
:10B3E000EE53FC4F982F9F5F8081809364099630C5
:10B3F00008F027C090934D0510925E090E946F5788
:10B4000081E080936109000000000000000000005E
:10B41000000000000000000000000000000000002C
:10B42000000000000000000000000000000000001C
:10B4300000000000000080916209809381098EBDA8
:10B44000089510924D05D8CF20915E09222309F06E
:10B4500045C00DB407FE42C084E080930004459AC5
:10B460003EB580914F0599278130910509F437C089
:10B47000823091050CF451C0029709F439C0209133
:10B480006109203208F030C045980000000000003B
:10B4900000000000000000000000000000000000AC
:10B4A000000000000000000000000000000000009C
:10B4B00000000000000000000000E0915F09F09132
:10B4C0006009E20FF11D80818EBD8091810990811C
:10B4D000890F809381092F5F209361090895353585
:10B4E00051F120934F05CBCF81E080935E09F3CFDC
:10B4F00080918309E82FFF27ED55F64F30838F5F4A
:10B50000809383098A3100F180915005381711F139
:10B510002093840910924F05B2CF892B09F0AFCF49
:10B520002093830930935005313809F0A8CF81E08A
:10B5300080934F05A4CF80915005830F80935005D1
:10B5400082E080934F059BCF80915005830F8093BD
:10B55000500595CF8AE1E3EAF9E0A9E8B9E0019066
:10B560000D928A95E1F781E08093840910924F054E
:10B5700086CF20E030E0882321F080915105882398
:10B5800081F48091580499278071907095958795E2
:10B5900095958795959587952817390791F0429A43
:10B5A000089521E030E080915804992780719070CF
:10B5B000959587959595879595958795281739073A
:10B5C00071F74298089520E030E0882321F08091BF
:10B5D0005105882391F480915804992780729070C6
:10B5E0009595879595958795959587959595879543
:10B5F0002817390729F0439A089521E030E0EBCF6E
:10B600004398089587B18C6087B9109252051092C3
:10B61000510580E00E94B95A80E00E94E35A1092DE
:10B62000580580E88093C903109255058093C8039C
:10B6300008958091590581508F3FB9F18093590544
:10B640003091560540E0332389F09091590580915F
:10B650005705981740F18091A908282F332780912A
:10B6600026039091270382179307ECF0842F0E9402
:10B67000B95A40E080915305882309F411C1909193
:10B68000590580915405981760F08091A908282FDA
:10B6900033278091260390912703821793070CF09C
:10B6A000FFC041E0FDC041E0E1CF89E08093590552
:10B6B00020915804822F992781FD30C080FFBFC0A0
:10B6C00030916D04332371F580919208E82FFF27A4
:10B6D000EE0FFF1FE25AF74F808191818C5A9F4FE6
:10B6E0000CF18081918185359105E4F48091930876
:10B6F000E82FFF27EE0FFF1FE25AF74F808191815D
:10B70000855B9F4F1CF481E080935205808191817D
:10B710008C3491053CF03093520504C080916D0447
:10B7200080935205E0915205422F5527BA0164706B
:10B73000707042FF19C08091A908282F332780918B
:10B740002603909127038217930774F443FD79C071
:10B75000E0935105809159056F5F7F4F99270E94B3
:10B76000AD656093590502C0E09351059091C708FB
:10B770009B3F08F43FC080911809873ED8F1909113
:10B78000C608392F3078309356058091C903892334
:10B7900029F080910D0967E10E948D65809357051E
:10B7A0009091C9089B3FB8F080914B09873E98F073
:10B7B0009091C808892F8078809353052091C80301
:10B7C000892F822329F08091110967E10E948D65FC
:10B7D0008093540537CF9B3FE0F080914B098A302E
:10B7E000C0F480E09091C80897FDE6CF81E0809397
:10B7F0005305E4CF9B3FB8F0809118098A3098F444
:10B8000080E09091C60897FF81E0382F309356056D
:10B81000BCCF8091550581508F3FB9F0809355057D
:10B820009091C808CBCF8091580581508F3F09F186
:10B83000809358059091C60830915605A6CF81E0B7
:10B840006FCF81E08093510585CF80914B09815066
:10B85000809355058091C8038130F1F08695282F9B
:10B860008093C8039091C808892F82238093530541
:10B87000A7CF809118098150809358058091C90302
:10B88000813061F086958093C9039091C608392F65
:10B890003823309356057BCF80E8E1CF80E8F3CFA3
:10B8A000842F0E94E35A08958091C9008F77809376
:10B8B000C9008091C9008F7B8093C9008091C90025
:10B8C0008F7D8093C9005A9A52981092CD0084E1DE
:10B8D00090E08093CC008091C80082608093C80083
:10B8E00080E18093C9008091CA008F778093CA005D
:10B8F0008091CA008F7B8093CA008091CA008F7D9F
:10B900008093CA008091CA008F7E8093CA00809184
:10B91000CA00877F8093CA008091C9008B7F809383
:10B92000C9008091CA0084608093CA008091CA00D7
:10B9300082608093CA008091C80087FF0CC080910C
:10B94000CE008091C800882334F48091CE0080918D
:10B95000C8008823A4F38091C90080688093C9003F
:10B9600008951F93CF93DF9380E197E20E94CE1456
:10B97000EC0110E08091C9008F778093C90080911D
:10B98000C9008F7E8093C9005A988EE597E09F93F7
:10B990008F931F930E9456110F900F900F90CE011E
:10B9A0000E94D714882309F066C04A9BF8CF8AE525
:10B9B00090E00E94CE14EC0184E997E09F938F936E
:10B9C0001F920E945611529A0F900F900F90CE0125
:10B9D0000E94D7148823D9F383E690E05A9A0197FE
:10B9E00097FFFCCF8FE891E05A98019797FFFCCF23
:10B9F00089E090E05A9A019797FFFCCF89E090E0A8
:10BA00005A98019797FFFCCF8FE891E05A9A0197D7
:10BA100097FFFCCF8FE891E05A98019797FFFCCFF2
:10BA200089E090E05A9A019797FFFCCF89E090E077
:10BA30005A98019797FFFCCF8FE891E05A9A0197A7
:10BA400097FFFCCF8FE891E05A98019797FFFCCFC2
:10BA500089E090E05A9A019797FFFCCF89E090E047
:10BA60005A98019797FFFCCF8FE891E05A9A019777
:10BA700097FFFCCF0AC08AE997E09F938F931F93AB
:10BA80000E9456110F900F900F9052985A980E9452
:10BA9000545CDF91CF911F9108951F920F920FB6C2
:10BAA0000F921124EF92FF920F931F932F933F93C6
:10BAB0004F935F936F937F938F939F93AF93BF93B6
:10BAC000CF93DF93EF93FF930091CE008091CA0351
:10BAD0009091CB03019709F45EC08091620590912B
:10BAE00063050E94D714482F552760915A0570911D
:10BAF0005B0561157105E9F16130710509F4EAC072
:10BB00006230710509F4EDC06330710509F45CC061
:10BB100081E090E09093CB038093CA0310925D057F
:10BB200010925C05109261051092600580915C0591
:10BB300090915D054097A0F080916005909161051E
:10BB4000892B11F41092830310925D0510925C050D
:10BB5000109261051092600510925B0510925A05D3
:10BB600087E090E00E94CE14909363058093620575
:10BB7000FDC0452BD9F281E090E090935B05809366
:10BB80005A0580915C0590915D05019690935D0545
:10BB900080935C05CBCF1092CB031092CA0387E051
:10BBA00090E00E94CE1490936305809362051092FA
:10BBB0005D0510925C0510925B0510925A0510927B
:10BBC0005F0510925E05D2C0452B09F0A1CF82E03F
:10BBD00090E090935B0580935A0580915C0590916D
:10BBE0005D05019690935D0580935C0580915E05EF
:10BBF00090915F05FC01F695E795F695E795EF7056
:10BC0000F0703196982F8827202F3327822B932B83
:10BC10009370805092400E94AD65EB30F10508F0C2
:10BC200085CF7F01EE0EFF1EF701E25AF74F8081AC
:10BC300091819B01281B390BC90137FD90C00697E4
:10BC400054F480917604883C08F087C08091760493
:10BC5000865F80937604F701E25AF74F80819181E5
:10BC60009C01220F331F280F391F260F371F37FD66
:10BC70007AC0E901D595C795D595C795CB010196B1
:10BC80008C179D070CF05CC0219780917604843B53
:10BC900008F450C087010C58174FF701E25AF74FCC
:10BCA00080819181FE01E81BF90BCF0163E070E018
:10BCB0000E94AD65CB01880F991F860F971FF80171
:10BCC000918380832EE538E0E20EF31EF701D183E5
:10BCD000C0832CCF4115510509F012CF82E090E0CE
:10BCE0004CCF4115510509F00FCF802F9927909324
:10BCF0005F0580935E0520915C0530915D052230E3
:10BD0000310569F083E090E090935B0580935A05DC
:10BD10002F5F3F4F30935D0520935C0507CF8091E7
:10BD20005E0587FF15C081E090E0909361058093E8
:10BD30006005E8CFF701EC58F74F11821082C2CFAF
:10BD400061507040C617D7070CF09FCF21969DCF4A
:10BD50005093610540936005D5CF88EC7ACF9095DC
:10BD600081959F4F6CCF2D5F3F4F83CFFF91EF9118
:10BD7000DF91CF91BF91AF919F918F917F916F9103
:10BD80005F914F913F912F911F910F91FF90EF90F5
:10BD90000F900FBE0F901F90189510926805089590
:10BDA0000E94CD5E089580916B0490916C049093F5
:10BDB0006A048093690480918A0490918B04A09115
:10BDC0008C04B0918D04B7FF04C081589F4FAF4FD2
:10BDD000BF4F27E0B595A795979587952A95D1F7F9
:10BDE00090936705809366050895209169043091CA
:10BDF0006A04280F311D30936A04209369048091EE
:10BE00008A0490918B04A0918C04B0918D04B7FFAB
:10BE100004C081589F4FAF4FBF4F37E0B595A795EE
:10BE2000979587953A95D1F7909367058093660526
:10BE3000089581E0809368050895CF93DF93409142
:10BE4000690450916A04509303084093020860E02B
:10BE500070E080916805882321F080918304882315
:10BE600029F07093650560936405A7C080916B0409
:10BE700090916C04841B950B209198033327289F85
:10BE8000A001299F500D389F500D11249A0157FD94
:10BE900079C0B90175956795759567958091160478
:10BEA0009091170497FD87C095958795860F971FEA
:10BEB0009093650580936405C0918A04D0918B04AA
:10BEC000E0918C04F0918D04F7FD70C067E0F5956A
:10BED000E795D795C7956A95D1F7809166059091BA
:10BEE0006705AA2797FDA095BA2FC81BD90BEA0BA7
:10BEF000FB0B80919703282F332744275527BE013A
:10BF0000CF010E946E6597FD4CC055E095958795D1
:10BF1000779567955A95D1F751E069317507ACF17E
:10BF200088E191E090936A0580936905209164050A
:10BF3000309165058091690590916A05280F391F38
:10BF400080915C049927829FA001839F500D929F4E
:10BF5000500D1124CA0162E370E00E94AD6580912A
:10BF60005B049927880F991F880F991F90958195D9
:10BF70009F4F681779070CF074CF909365058093F5
:10BF800064051BC02D5F3F4F84CF4EEF683E7407A2
:10BF90001CF488EE9EEFC6CF70936A056093690526
:10BFA000C5CF615E7F4F8F4F9F4FAFCFC158DF4FDF
:10BFB000EF4FFF4F8BCF019677CF80916405909123
:10BFC00065059093090880930808DF91CF91089543
:10BFD000CF93DF938091980880FF12C081E0809317
:10BFE0006B05E091DB03F091DC03EF3FF10589F095
:10BFF00080916B059927009751F10197D1F52EC0DB
:10C0000010926B05E091DB03F091DC03EF3FF1054B
:10C0100079F784EF91E00E94CE14EC01CE010E94EA
:10C02000D7148823D9F380919208E82FFF27EE0FC9
:10C03000FF1FE25AF74F0190F081E02DF093DC03EF
:10C04000E093DB0380916B0599270097B1F6EC5ADA
:10C05000FF4F7CF082E080936B050BC0F7FD05C0BD
:10C060003597C4F70E945D6004C0F095E195FF4FDD
:10C07000F7CFDF91CF91089580919208E82FFF27A5
:10C08000EE0FFF1FE25AF74F8081918190930708CE
:10C090008093060888589F4F089580916B059927D3
:10C0A000009729F0019731F080E090E008950E9418
:10C0B0003C6008950E9479600895AAE0B0E00E9473
:10C0C000FD65802D992780936E05982F80915D04E2
:10C0D000989FC001112464E670E00E94AD656093F2
:10C0E0006D05ACE0B0E00E94FD65802D80936C058D
:10C0F0000895FF920F931F93CF93DF93F0909208D0
:10C10000EF2DFF27EE0FFF1FE25AF74FC081D181BD
:10C110008091DB039091DC03C81BD90B80916D04E7
:10C12000882309F44BC01C161D060CF0F6C09E01B6
:10C13000442737FD4095542FCA01B9010E946E650E
:10C14000DC01CB01BC01CD0126E930E040E050E04C
:10C150000E94E2658E01020F131F053011050CF4D9
:10C160006FC0A0917905B0917A05A8014A0F5B1FB5
:10C170004450504080917B0599278930910509F4FE
:10C1800074C08A3091050CF096C08530910509F491
:10C190007BC1863091050CF015C18330910509F4FF
:10C1A00014C2843091050CF0CDC2509378054093B1
:10C1B0007705019709F451C2BA0113C010927605B0
:10C1C00010927505109278051092770510927A05F5
:10C1D0001092790500E010E081E080937B05D801A2
:10C1E000B80120917105309172054091750550910B
:10C1F0007605CB01841B950B281739070CF4C90170
:10C20000309521953F4F821793070CF4C901209177
:10C210006F05309170052115310549F4840F951F84
:10C22000909376058093750525E030E0AC012150B0
:10C2300030403093700520936F0557FF55C334C0CD
:10C240002FEF0C3F12070CF062C0A0917905B0915E
:10C250007A05A8014A0F5B1F4C5F5F4F80917B05F9
:10C2600099278930910509F08CCF50937805409338
:10C270007705EF2DFF27EE0FFF1FE25AF74F808162
:10C2800091818C5A9F4F0CF45FC084E690E09093AC
:10C290007D0580937C052396279708F4F7C160916C
:10C2A0007705709178059DCF1092760510927505EF
:10C2B00040E050E019C38D30910509F4B5C08E30CF
:10C2C00091050CF051C08B30910509F459C10C97C0
:10C2D0000CF06FC220917E0530917F052A0F3B1F25
:10C2E000309378052093770580917C0590917D05AA
:10C2F000019790937D0580937C05892B19F488E044
:10C3000080937B0524970CF485C2B9016ACFA09174
:10C310007905B0917A05AD012DCF9E01442737FDF7
:10C320004095542FCA01B9010E946E65DC01CB0112
:10C33000BC01CD0126E930E040E050E00E94E2651A
:10C340008E01021B130B09CF80917C0590917D0516
:10C35000019790937D0580937C05892B09F09BCFF5
:10C360008EE080937B0597CF8F30910509F44CC107
:10C370008F3091050CF404C25093780540937705F3
:10C38000409709F019CF80916E059927BA01481797
:10C3900059077CF024E130E0309372052093710559
:10C3A0008CE080937B0584EF91E09093020480936E
:10C3B0000104CE01D7FD93C205970CF412CF0E9461
:10C3C000CD5E44C050937805409377058730910542
:10C3D00009F4C7C008970CF069C1C530D1050CF449
:10C3E000FEC180916D05282F332730937A05209365
:10C3F0007905C135D1054CF08FE080937B0584EF42
:10C4000091E090930204809301046091770570910C
:10C410007805261737070CF00AC230937805209369
:10C420007705D901BD01DDCEB0937805A0937705DE
:10C430009E01D7FD0EC125303105A4F30E94CD5ECB
:10C4400084EF91E0909302048093010420916405AD
:10C450003091650537FD10C235952795359527959F
:10C460008091790590917A05821B930B90937A05C0
:10C4700080937905909378058093770529E0209340
:10C480007B05DC01BD01ADCE509378054093770567
:10C4900020919108E22FFF27EE0FFF1FE25AF74F7E
:10C4A000808191818C5E9F4F0CF442C0E22FFF2768
:10C4B000EE0FFF1FE25AF74F808191814597ACF054
:10C4C00080916C05882389F0815080936C05ACE0E5
:10C4D000B0E0082E0E940A6684EF91E09093020477
:10C4E0008093010484E080937B0520917305309153
:10C4F0007405253031058CF0201B310B80916C05C3
:10C500009927281739074CF084E080937B0584EF46
:10C5100091E09093020480930104109278051092A8
:10C520007705A0917905B0917A0560E070E059CE69
:10C5300080916C05843108F0B9CF8F5F80936C05D2
:10C54000ACE0B0E0082E0E940A6684EF91E0909380
:10C5500002048093010484E080937B05209191087C
:10C56000A5CFC530D1050CF45AC12AE030E0309394
:10C5700072052093710588E080937B05BA0135CE62
:10C5800050937805409377052396279708F00DC1BF
:10C5900080917305909174059801281B390BC9018E
:10C5A0000196039708F001C180917C0590917D056B
:10C5B000019790937D0580937C05892B09F0FCCD34
:10C5C0008CE080937B05BA010CCE509378054093A4
:10C5D0007705BA0150937605409375052A976CF05C
:10C5E00080917305909174059801281B390BC9013E
:10C5F00037FD71C102970CF41CC182E390E0909367
:10C600007D0580937C05EDCD5093780540937705AB
:10C6100080916D05282F3327BA01241735072CF494
:10C620003093780520937705B901C430D10554F4CF
:10C63000CC5FDF4F1CF48EE080937B05621773079D
:10C640000CF024C125E030E0309372052093710591
:10C65000CCCD309521953F4FEECE80919108E82FBB
:10C66000FF27EE0FFF1FE25AF74F80819181873439
:10C6700091050CF404C183E080937B0584EF91E085
:10C680009093020480930104BA01ABCD0E94D35E63
:10C6900089E190E090937D0580937C058BE0809309
:10C6A0007B05A0917905B0917A05F9CDEF2DFF2793
:10C6B000EE0FFF1FE25AF74F808191818C5A9F4FF6
:10C6C0000CF498C084E690E090937D0580937C05FF
:10C6D0004091730550917405453051054CF09A0115
:10C6E000201B310B80916C0599272817390744F4DA
:10C6F000443051050CF0D3CD8091C50882FFCFCDD9
:10C700000E94D35E809173059091740590937F058C
:10C7100080937E058AE080937B0589E190E0909389
:10C720007D0580937C0524E130E0309372052093F1
:10C730007105A0917905B0917A05609177057091A6
:10C74000780553CD04301105A4F480919108E82FA9
:10C75000FF27EE0FFF1FE25AF74F80819181019072
:10C76000F081E02DF7FDB3C034971CF485E0809391
:10C770007B05109278051092770560E070E031CD6E
:10C7800022E030E0309372052093710510927A0513
:10C7900010927905109278051092770586E08093C3
:10C7A0007B05A0E0B0E0BD0120CD89E080937B0552
:10C7B00076CD509378054093770550937605409356
:10C7C000750550937A05409379050E94195F84EFAF
:10C7D00091E090930204809301048DE060CF8091FA
:10C7E0006D0599278A179B0709F059CD87E080933B
:10C7F0007B0555CD80917C0590917D0501979093A7
:10C800007D0580937C05892B09F062CF8EE08093B3
:10C810007B055ECF30937A0520937905D6CFCC5F28
:10C82000DF4F0CF0C9CC8EE080937B05CCCED901D4
:10C83000D8CC80917C0590917D05019790937D05E2
:10C8400080937C05892B09F0CCCC80916E059927CB
:10C850008617970709F4C5CC8091750580936E05FE
:10C86000AAE0B0E0082E0E940A6684EF91E090935F
:10C8700002048093010415CF2D5F3F4FEDCD8081E1
:10C8800091818A5B9F4F7CF684E0F6CE80916E05A5
:10C89000992790937A058093790525E030E03093CD
:10C8A0007205209371050E94D35E80919B080E94BF
:10C8B000F55E0E94195F80E180937B05A091790568
:10C8C000B0917A056091770570917805BBCEF095AF
:10C8D000E195FF4F49CF909581959F4F8BCE88274B
:10C8E00099278C1B9D0B68CD1093740500937305DD
:10C8F000B0930508A0930408109307080093060856
:10C90000CA01DF91CF911F910F91FF900895FC0113
:10C910004150504030F001900616D1F73197CF01C9
:10C9200008958827992708955058192EA6D001D028
:10C930008CC0BA176207730784079507B1F188F4B2
:10C940000EF410940B2EBA2FA02D062E622F202D40
:10C95000072E732F302D082E842F402D092E952F52
:10C96000502DFF275523B9F0591B49F0573E98F039
:10C97000469537952795A795F0405395C9F776F0DA
:10C98000BA0F621F731F841F30F4879577956795E0
:10C99000B795F040939517FA0F2E0895BF1BBB274C
:10C9A000BA0B620B730B840BF6CFDEF692C097FBCB
:10C9B00070D09F3738F0FEE9F91B982F872F762F1C
:10C9C0006B2F05C083C09695879577956795F15035
:10C9D000D0F73EF490958095709561957F4F8F4F7D
:10C9E0009F4F0895E89403C097FB0EF4F3DFB62F32
:10C9F000672F782F892F9EE9002427C00ED05EF084
:10CA000004C00BD026F001C008D019F020F48FEF3D
:10CA1000089580E0089581E0089597FB092E05268A
:10CA200000F868942DD0E89407FC07C062177307DC
:10CA30008407950721F008F40094079498940895CA
:10CA40009A95BB0F661F771F881F11249923A1F0A9
:10CA50008823B2F79F3F59F0BB0F48F421F4002020
:10CA600011F460FF04C06F5F7F4F8F4F9F4F881F8F
:10CA70009795879597F9089529C0052E092607FAF5
:10CA8000440F551F5F3F79F0AA27A51708F051E022
:10CA90004795880F991F9F3F31F0BB27B91708F0C2
:10CAA00091E0879508959F919F91112414C097FB61
:10CAB000880F991F9F3F31F0BB27B91708F091E00D
:10CAC000879508959F919F91112405C06627772728
:10CAD0008827992708959FEF80EC0895629FD001E1
:10CAE000739FF001829FE00DF11D649FE00DF11D29
:10CAF000929FF00D839FF00D749FF00D659FF00DD8
:10CB00009927729FB00DE11DF91F639FB00DE11DC4
:10CB1000F91FBD01CF0111240895991B79E004C0CC
:10CB2000991F961708F0961B881F7A95C9F780956C
:10CB30000895AA1BBB1B51E107C0AA1FBB1FA61764
:10CB4000B70710F0A61BB70B881F991F5A95A9F7B6
:10CB500080959095BC01CD01089597FB092E07267D
:10CB60000AD077FD04D0E5DF06D000201AF47095D6
:10CB700061957F4F0895F6F7909581959F4F0895A1
:10CB8000A1E21A2EAA1BBB1BFD010DC0AA1FBB1FD1
:10CB9000EE1FFF1FA217B307E407F50720F0A21B43
:10CBA000B30BE40BF50B661F771F881F991F1A94B0
:10CBB00069F760957095809590959B01AC01BD01DA
:10CBC000CF01089597FB092E05260ED057FD04D0FE
:10CBD000D7DF0AD0001C38F4509540953095219548
:10CBE0003F4F4F4F5F4F0895F6F7909580957095A2
:10CBF00061957F4F8F4F9F4F0895F999FECFB2BD3A
:10CC0000A1BDF89A119600B40895F7DF01921A9425
:10CC1000E1F70895F999FECFB2BDA1BD00BC119610
:10CC20000FB6F894FA9AF99A0FBE08950190F2DFC0
:06CC30001A94E1F70895DB
:10CC3600010A0151756164726F0000416E676C658F
:10CC46004E69636B20202020202020416E676C6592
:10CC5600526F6C6C202020202020204163634E6997
:10CC6600636B202020202020202020416363526F08
:10CC76006C6C2020202020202020204779726F47CE
:10CC8600696572202020202020202048696768746A
:10CC96002056616C756520202020204163635A2050
:10CCA60020202020202020202020204761732020C3
:10CCB6002020202020202020202020436F6D70611E
:10CCC60073732056616C7565202020566F6C7461F5
:10CCD6006765202020202020202020456D70666179
:10CCE6006E672020202020202020204779726F2088
:10CCF6004B6F6D70617373202020204D6F746F72BF
:10CD06002046726F6E7420202020204D6F746F7243
:10CD160020526561722020202020204D6F746F7292
:10CD2600204C6566742020202020204D6F746F7281
:10CD3600205269676874202020202020202020208F
:10CD460020202020202020202020202020202020DD
:10CD560020202020202020202020202020202020CD
:10CD660020202020202020202020204D4B334D61E4
:10CD7600672043616C537461746520536572766FE6
:10CD8600202020202020202020202020202020209D
:10CD9600202020202020202020202020202020208D
:10CDA600202020202020202020202020202020207D
:10CDB6002020202020202020202020536F6C6C482B
:10CDC6006F656865202020202020205069746368E4
:10CDD6004F66667365742020202020537469636B48
:10CDE60056616C75652020202020204B616C6D619A
:10CDF6006E5F4D6178447269667420202020202081
:10CE060020202020202020202020204E617669200E
:10CE160053657269616C20446174614750535F4E7B
:10CE260069636B20202020202020204750535F522A
:10CE36006F6C6C2020202020202020C8000164FF79
:10CE460001FFFF01FC01FC0101737373FF03007D09
:10CE56000000C409C40964000F48616C6C6F205758
:10CE6600656C740000000000000000000000000077
:10CE760000000000000000000000000000000000AC
:10CE8600000000000000000000000000000000009C
:10CE9600000000000000000000000000000000008C
:10CEA6000000000000000000000102030405060760
:10CEB60008090A01040B050000ECFF6440415A46CC
:10CEC600640A02969608403A10FB30380190D00367
:10CED6000090D00300F401640053706F7274000078
:10CEE6004E6F726D616C0000426567696E6E6572A9
:10CEF60000000A0B0D0B0C0E010101004D4B004DFD
:0ECF060044003F3F00CC03CF03D203FF0000E6
:00000001FF
